:020000040800F2
:103000000080002093C8000811C200084DC20008CB
:1030100000000000000000000000000000000000B0
:103020000000000000000000000000009BC9000834
:1030300000000000000000009DC900085D020020A3
:1030400065C8000867C8000869C800086BC80008A0
:103050006DC800086FC8000871C8000873C8000870
:1030600075C800086D02002077C8000879C80008FC
:10307000E10200207BC800087DC800087FC8000866
:1030800081C80008ADC20008BDC20008CDC200085A
:10309000DDC20008EDC20008FDC2000883C80008B8
:1030A00085C8000887C8000889C8000849030020AF
:1030B0008BC800088DC800088FC8000891C8000898
:1030C000014802490160704708ED00E00030000847
:1030D000B0B51E4D2C1F20688006400F411E0329ED
:1030E00022D81B487944097949008F442301171AD3
:1030F000296803220A40032A00D016482968490695
:10310000490F491C09F09AF929684904490E4843B6
:103110002968490F491C09F091F90BE07D20000254
:1031200008E00120C00305E00C3D28688004410F41
:103130000848C84008494860226892093C23134067
:10314000064AD258D0404860B0BDC0460C1002407C
:1031500000127A000024F400E40500205CC7000897
:10316000F0B585B0804D2F68B8680224400728D498
:103170005426A85D012824D001200390A855F868A2
:10318000C0077A4B0BD1B868C00704D0B8681840A4
:1031900002210143B960F86801210143F96000246C
:1031A0000494B868C00742D118462F30B96801426C
:1031B0000AD0A86D10210143A965E86D01242043C0
:1031C000E865204605B0F0BDB868184001210291BD
:1031D0000843B86066480068000200D59CE0687E3D
:1031E000012824D0654841683A68D2071FD101946C
:1031F00002E03A68D2071AD1BA68D2070FD1BA688A
:103200001A4034462E461D460B460146029802439C
:10321000084619462B4635462646019CBA60426848
:10322000521A032AE5D33A68D207E2D1C1E7AC5576
:10323000A86D534901402846039D2A02029289182D
:103240008165C4651C233B60016D4E4A4E4E4F485C
:10325000C8620E634A637868102202437A602420B1
:10326000085C012801D102244BE00A462432157083
:103270005078012841D102205070CC630A68106850
:103280000125A8431060886CCE6C4660086D0090E4
:10329000002802D0486D8E6D46604037086C18409B
:1032A0000395012383403A4806681E4306600620C2
:1032B00050608B683748102B06462B4D00D03E4699
:1032C0009660102B00D00746D76010680E2303438A
:1032D0001360496C0868C003029E02D50868304339
:1032E000086000990029214B02D00868304308602B
:1032F000106803990843106005E014708020C863CB
:103300002C461A4B184D28688168194004220A433C
:103310008260204605B0F0BD16484068164909F0A5
:103320008DF8124B401C04900498002800D156E7F9
:103330000498401E04900498002800D14FE7049898
:10334000401E04900498002800D148E70498401ECD
:1033500004900498002800D141E70498401E04908E
:1033600004980028E4D13AE71C120020E8FFFF7F10
:1033700008270140E4050020400D0300A8110020AB
:10338000FEF0FFFF9FC90008FFC8000899C80008A9
:0833900004000240F0110020CE
:10339800F0B587B00025069554269E4FB95D0129E2
:1033A80002D1022007B0F0BD0124BC5539688A68F3
:1033B800520714D43B694268022A18D104221343E5
:1033C800964A93426FD1944AD3430268D043184334
:1033D8008B6A03408B620024002A68D4CCE0B86D65
:1033E80020210143B965BD55012007B0F0BD059204
:1033F80004273B43884A894CA34265D1046822408C
:103408008B6A13438B62834F22024B699343806814
:103418001040834A02401A434A6122460024002A87
:1034280000D4A9E0012005907E48036807208005A4
:103438001946049001407C480292824200D082E002
:103448000598C0051A4602407DD1764A1268049B49
:103458009A431143014373480160764840687649AE
:1034680008F0E8FF0C2141430C310691069800282A
:1034780000D181E00698401E0690069800287BD06F
:103488000698401E06900698002875D00698401E9B
:103498000690069800286FD00698401E0690069859
:1034A8000028E7D168E002680024002A64D55D4856
:1034B80001685E4B9A4266D05D4B9A4266D05A4B81
:1034C8009A4259D105225FE002971F24059B1C40B0
:1034D8000F2300930494A3404E4F3C6E01939C43EA
:1034E80023460468144203934AD0E2072A465FD170
:1034F800A20758D4620758D4220758D4E206029A81
:1035080056D4A2066CD462066CD422066CD4E205AA
:103518006CD40294A2056BD462056BD422056BD4DB
:10352800E2046BD4A2046BD462046BD42204009A24
:10353800384F3DD4E20368D4A20368D46203D3179A
:1035480012221A405FE03948029A824204D1059853
:1035580000061A46024007D03548029A82420BD12B
:1035680005988005034007D12E4A1268049B9A43A8
:10357800114301432B4811E0BD55204607B0F0BD6B
:103588006200D20E14E00322920501E00322D20564
:103598001140072292050368934359180160BD55ED
:1035A800002007B0F0BD012202E0022200E0032261
:1035B800049B9A40039B1A433A66059A9208FB6952
:1035C800934200D820E7019AD2438B6A13400593AF
:1035D800A200120F049B9A40059B1A438A6213E7C4
:1035E8000522E5E70622E3E70722E1E70822DFE70D
:1035F800092208E00A2206E00B2204E00C2202E07D
:103608000D2200E00E22034FD2E71022FBE7112221
:10361800F9E7C0461C120020FFFF070004000080E5
:1036280000FFFF0708270140001000B0004000B865
:0C363800002000B4E4050020400D030059
:10364400F0B583B05422C44FB95C012902D10220E1
:1036540003B0F0BD39688C686407C04B00D58EE0B8
:10366400066844689E4215D10125EE05B44266D031
:103674000326B605B4426BD11F24A40687682740ED
:10368400CB680293BA4C1C403C19B34FB34BA419FA
:10369400CC6061E00127FD05AC42B14B7FD00297BD
:1036A4000325AF05BC4200D089E00C46A034009449
:1036B4008768AE4C01973C409E42A74F00D08CE0F7
:1036C400002C00D1C0E0019BDC0700D0C4E09C07C3
:1036D40000D5CBE05C0700D5CAE01C0700D5C8E0E4
:1036E400DC0600D5FEE09C0600D5FFE05C0600D5B4
:1036F40000E11C0600D501E1DC0500D502E19C05D2
:1037040000D503E15C0500D504E11C0500D505E105
:10371400DC0400D506E19C0400D507E15C0400D577
:1037240008E11C0400D509E1DC0300D50AE19C038F
:1037340000D50BE15C03E4171225254007E1CC68B2
:103744003B468B4F2740BC191F46844BCC6003E09B
:10375400CC68874E2640CE602C04BD6DA543BD6564
:1037640080240C604D68067B012E06D125434D60F4
:10377400066905689D4207D0A0E0A5434D6006692F
:1037840005689D4200D099E0CB689B08062423403D
:103794009E40CB689B08234044699C408FE0714C59
:1037A400E443F5432543F40C04272740CC19A02710
:1037B400E3592B406C4D35401D43E5510BE0694BFB
:1037C400DB43F4431C43F30C04251D404B19A02593
:1037D4005E5926405E51604F51E0002C38D0019B69
:1037E400DC073BD19C07029E39D45C0778D41C07C4
:1037F4002E4634D4DC0677D49C0679D45C067BD47C
:103804001C067DD4DC057FD49C0500D580E05C05D6
:1038140000D581E01C0500D582E0DC0400D583E0FE
:103824009C0400D584E05C0400D585E01C0400D52C
:1038340086E0DC0300D587E09C0300D589E05C03C7
:10384400E4171226264085E0019B5C00E50E10E09B
:10385400019B5C00E60E02E000250AE00026029DC2
:10386400B540009B5C682C435C6008E0012500E0E7
:1038740002250124AC40009B1D6825431D60BC6DDE
:103884000368374DAB4205D101235D04AC43BC65ED
:103894001C0204E001239D04AC43BC655C020C6083
:1038A4004D68037B012B01D1254300E0A5434D6006
:1038B4002A4B066905689D4200D165E744690020EA
:1038C400B85432042243AB02DC0F9B0F1B199B003C
:1038D400C9180B6A274C1C4014430C6203B0F0BD9A
:1038E4000226BCE70425C4E70426B8E70525C0E79B
:1038F4000526B4E70625BCE70626B0E70725B8E7A2
:103904000726ACE7082522E0082623E009251EE067
:1039140009261FE00A251AE00A261BE00B2516E0FB
:103924000B2617E00C2512E00C2613E00D250EE003
:103934000D260FE00E250AE00E260BE00F2506E00B
:103944000F2607E0102502E0102603E01125024FA0
:103954008FE71126004F82E71C1200200000C07C74
:10396400FFFF1700FFFFC77CFFFF8700FFFF070073
:08397400FFFF3F8300F000F0AB
:10397C00F0B582B0654A537D012B02D1022002B012
:10398C00F0BD02231375012757750668042E1DD14F
:10399C00019600292CD014695D4E636B002B51D518
:1039AC007368012B46D8636B002B4BD57368012BC6
:1039BC0040D8636B002B45D57368012B3AD8636BE9
:1039CC00002B3FD57368022BE7D333E014690369EE
:1039DC00012B76D11023194043698B401F258D4054
:1039EC003246A66BAE431E43A6631646474A6AE0B0
:1039FC001469474E012377680093DD03636B2B42F8
:103A0C0035D07368DB1B012B14D8636B2B422ED083
:103A1C007368DB1B012B0DD8636B2B4227D07368AB
:103A2C00DB1B012B06D8636B2B4220D07368DB1B8E
:103A3C00022BE3D3106A0821014311620320107595
:103A4C0002B0F0BD0097756873685B1B012B0BD837
:103A5C0073685B1B012B07D873685B1B012B03D8A6
:103A6C0073685B1B022BEFD38369636412E0756888
:103A7C0073685B1B012B0BD873685B1B012B07D87E
:103A8C0073685B1B012B03D873685B1B022BEFD392
:103A9C008369236410250D40C369AB401D4EAE40B5
:103AAC00A76CB7431F43A764036AAB40FF26AE4025
:103ABC00E56CB5431D43E564009F019E0369012B32
:103ACC0088D01023194007238B40E56B9D438368F6
:103ADC003343C6681E438E402E43E663BB038B40C4
:103AEC0025689D432560406888400B4B8B402568BA
:103AFC009D4305432560C020884021688143216097
:103B0C0000205075177502B0F0BDC046C0070020EC
:0C3B1C00A8110020FF030000FE0F0000B5
:103B2800F0B583B000283FD004460646243602206C
:103B38007070276838683049014039602F488030F4
:103B4800A0642F483818142108F074FC80002B4911
:103B58004118206401916164F8B20838142108F012
:103B680069FC1F210140012528468840E064A268BD
:103B7800E168114323690B4361691943A3690B4346
:103B8800E1691943236A0B4339681943396002957F
:103B9800A9038A421B4A0AD1002301990B6063607A
:103BA80010601F461D461CE0012003B0F0BD63688D
:103BB8003F211940019D29601060581E00230328E9
:103BC8001F461D460DD8481E810053180021D9678D
:103BD80003210140029D8D400B4805607C33BC32B7
:103BE80017460020E06323656765A5653070029974
:103BF800717003B0F0BDC0460F80FFFF000802409F
:0C3C0800F8FFFDBF8408024044090240A0
:103C1400F0B585B056490C78002C02D0022005B0CE
:103C2400F0BD0290039301270F707D20C100514E17
:103C34007068049141183C044F4D2868204216D006
:103C4400736803208B426CD22B6823420FD07368B5
:103C54008B4266D22B68234209D073688B4260D2B0
:103C64002B68234203D073688B42E6D359E028685B
:103C740042494B1C01932B600842384651D170686D
:103C8400049941180120009087042868384216D00E
:103C9400736803208B4244D22B683B420FD0736875
:103CA4008B423ED22B683B4209D073688B4238D298
:103CB4002B683B4203D073688B42E6D331E06868DB
:103CC40000990843686002990A60BFF36F8F0398F4
:103CD40048607068049941182868204216D07268B8
:103CE40003208A4219D22A6822420FD072688A427B
:103CF40013D22A68224209D072688A420DD22A68F5
:103D0400224203D072688A42E6D306E02868019909
:103D140029601A490842009808D06968009A9143BA
:103D240069600021124A117005B0F0BD70680499F1
:103D340041182A6800203A42EFD0736803228B426C
:103D440013D22B683B42E8D073688B420DD22B68A8
:103D54003B42E2D073688B4207D22B683B42DCD0F3
:103D6400706888421046E4D3D7E70320D5E7C046FD
:103D74002C110020A811002010200240FAC30000DA
:103D8400F0B586B00246884C2078002802D0022084
:103D940006B0F0BD0491012323707D20C100834D42
:103DA4006868059146181F04814C2068384216D073
:103DB40069680320B1421AD2216839420FD0696878
:103DC400B14214D22168394209D06968B1420ED295
:103DD4002168394203D06968B142E6D307E020681C
:103DE40074494E1C039626600842184604D00021EC
:103DF4006D4A117006B0F0BD686805994618012037
:103E0400029083042068184216D069680320B142E6
:103E1400EDD2216819420FD06968B142E7D2216816
:103E2400194209D06968B142E1D22168194203D02C
:103E34006968B142E6D3DAE70420506010680428C8
:103E440020D1381D61680143616068680599421892
:103E54002068384270D0696803209142C7D2216833
:103E6400394269D069689142C1D22168394263D02C
:103E740069689142BBD2216839425DD06968914238
:103E8400E6D3B4E70026F043049908609168D0684B
:103E94004218914258D20096474E606830400191D2
:103EA400C9000143B81C0843606068680599461856
:103EB4002068384216D069680320B1426CD2216868
:103EC40039420FD06968B14266D22168394209D0BB
:103ED4006968B14260D22168394203D06968B1424D
:103EE400E6D359E02068039921603249084252D14F
:103EF4006868059946182068184216D06968032036
:103F0400B14249D2216819420FD06968B14243D203
:103F14002168194209D06968B1423DD22168194229
:103F240003D06968B142E6D336E00199491C914255
:103F3400214EB2D1009832E02068039921601D49D6
:103F4400084203D0012052E7002028E06868059960
:103F54004118226800201A4200D148E76E68032203
:103F64008E4216D226681E4200D140E76E688E4209
:103F74000FD226681E4200D139E76E688E4208D2FD
:103F840026681E4200D132E7686888421046E0D3B2
:103F94002DE703202BE702980499019A0A606168CF
:103FA40002229143616022E72C110020A811002015
:0C3FB40010200240FAC3000005FEFEFFD2
:103FC000F0B58CB006900B68002B00D1C6E06448B9
:103FD000069A824201D0052000E0032000900124CF
:103FE00000200246074603940B900A90019112E0CC
:103FF0001343059A5B4843600B681846E0400B9DED
:10400000AD1C0B95121D0837641C0A9E761C0A967F
:10401000002800D1A2E0601E039E09908640334034
:104020000793E9D00B9B08974D6803212F460F405B
:10403000781E01280592029519D804941C469940CF
:10404000069A90688843019BDB68A3400343936012
:10405000E806049CC00F099B98405368B34316467A
:10406000059A03437360CB430A9845000AE0032096
:104070001D469840C343032F069E03D104930B9D16
:1040800001991CE0F0680493184001998B68AB40DB
:104090000343F360022F12D11C2010400F278740EA
:1040A000099BDB089B00F3181E6ABE430F6987401B
:1040B0003743069E1F624B6803271F4000E0029BA8
:1040C000AF403068049D2840384330609803800F2B
:1040D000089F91D0182038400F2686400323099F5F
:1040E0009F43204AD7193B6EB343603705263607F6
:1040F000069AB2420AD01D4EB24205D01C4EB242C0
:10410000009E04D1022602E0012600E0002686403F
:104110001E433E60144806684868C30302D5079AE8
:10412000164301E0079A9643089F0F4B1E605E6896
:10413000830301D5164300E096430B4B5E60094BA9
:104140001E68C30201D5164300E09643054B1E606E
:104150005B68800200D54BE793434AE70CB0F0BDA3
:10416000000C00500018024080180240000400506B
:0441700000080050F3
:10417400F0B588B00121002216461746029100903E
:1041840024E0069DB5402B4C2068284320601C2069
:104194003840059A82400398C00880002018036ABA
:1041A40093430362A068A843A0606068079B984398
:1041B4006060E068A843E0600098049A0346CB403E
:1041C4000832B61C3F1D491C002B2DD04D1E029BEE
:1041D400AB401C460440F1D00793182004921040D1
:1041E4000F22059282400323039506939D430F4BB0
:1041F4005B1901931D6E1540012383409D42C0D17C
:10420400019D60350A4B1868A04318605868A043A4
:104214005860064B1868A04318605868A04358605B
:10422400286890432860ACE708B0F0BD001802404D
:08423400801802400004005054
:10423C00F0B586B00746036899038D4A03D4002075
:10424C00D90761D166E00497012528071446183C6C
:10425C0021680140039106D1216801432160216846
:10426C000140059105990194029000952E02814C14
:10427C00216831432160804F7D68216831421AD119
:10428C007968491B0320022933D82168314212D1A5
:10429C007968491B02292CD8216831420BD17968E5
:1042AC00491B022925D82168314204D17968491B60
:1042BC000229E2D91DE00320010294680C40049904
:1042CC000E6B10D0B4420BD0946800990904956819
:1042DC000D43956095688D43956068490C409460DA
:1042EC00E10700D09DE0906864490840304390603D
:1042FC0000200399002904D1019D2968029CA14347
:10430C002960049FD90705D011680324A1437C6858
:10431C000C43146099070BD4D90611D4990518D401
:10432C0059051FD4990626D4012459042DD43BE0F9
:10433C0011680C24A143BC680C431460D906EDD55C
:10434C000321890214688C43F96821431160990593
:10435C00E6D50321890414688C43B96921431160A3
:10436C005905DFD50321090514688C43F9692143EC
:10437C0011609906D8D50321090314688C43396957
:10438C0021431160012459040ED511683D4D29407B
:10439C003E6A31431160691C8E4205D121041546D9
:1043AC00483D2E680E432E60190305D51168402533
:1043BC00A9437D6A0D431560A50599020FD51168B7
:1043CC00A943BE6A31431160AE4208D12106039164
:1043DC001646483E049737680F433760049F2B42BC
:1043EC000CD025061168A943FE6A31431160AE4218
:1043FC0004D1114648390E682E430E6019050ED5AE
:10440C00A10303239B0315689D437B691D43156022
:10441C008B4204D12104483A13680B43136006B055
:10442C00F0BD7C68164D9168890700D55BE779680B
:10443C00091BA94200D95CE79168890700D552E7AE
:10444C007968091BA94200D953E79168890700D5FF
:10445C0049E77968091BA94200D94AE7916889079D
:10446C0000D540E77968091BA942DCD941E7C04671
:10447C005410024000700040A8110020FFFCFFFF08
:08448C0088130000FFFFFF3F51
:10449400F0B58FB0002824D0044606463C36707828
:1044A400002821D00220707021680D680120830744
:1044B400994205D0A74A914202D0A74A91425DD1C0
:1044C40070229543A2682A43A44DA9425ADD924B17
:1044D40099424CDC9F4B99425CD0934B994259D002
:1044E400A9E001200FB0F0BD307002A8001D3021FA
:1044F40008F028F92168874881427ADD864881429C
:1045040000DD9AE08748814200D1B4E086488142C8
:10451400C8D10127B805029002A8FFF78DFE002834
:1045240013D08749002008F0DFF88649002008F0FE
:10453400DBF88549002008F0D7F88449002008F00A
:10454400D3F88349002008F0CFF8380479490A6881
:1045540002430A6009680140019101987648416864
:10456400FF22914341603805744908609AE76C4B17
:1045740099420FD0694B99420CD05CE02A46774DA2
:10458400A942A4DC994205D0734B994202D0654BF1
:10459400994250D103231B029A43256915432346AC
:1045A4003E33224644328027BD43A7692F430F6020
:1045B400E568CD6265688D62694D4D190A27FD4134
:1045C400072D06D80746AF40E1252F4201D0646984
:1045D4000C6348611071187058709870D870187115
:1045E4005871107050709070D070707000200FB0BF
:1045F400F0BD01208207914254D04C4A91425BD0D5
:104604004B4A914200D04DE74A49091F0A682023CA
:104614001A430A600968194001910199FF210904AC
:10462400454A13688B430321890559181160800496
:104634004249086036E71546B1E73848814252D00E
:104644003748814200D02DE701208104394A13689C
:104654000B43136012680A4001920199FF21090477
:10466400354A53688B4303218905591851608005E5
:104674003249086016E70120C1032E4A13680B4330
:10468400136012680A4001920199FF2109062A4A1F
:1046940013688B430321890759181160C004274903
:1046A4000860FFE62349091F0A6802430A60096893
:1046B400014001910198F5E61E49091F0A6810237B
:1046C4001A430A600968194001910199FF210902FE
:1046D400194A13688B430321890359181160400454
:1046E40016490860DEE601204104124A13680B43B0
:1046F400136012680A4001920199FF2109020E4ACF
:1047040053688B43032189035918516040050B49B1
:104714000860C7E6FF1F0040FF430140004401401A
:1047240000480140002000400040014000100040CB
:10473400001400404010024010E400E000E100E0FA
:10474400C0D200085ED000083DC800082DCD000886
:104754002CD00008002C014000040040FF2B014035
:0447640000D4FEBFC0
:10476800F0B583B004460120C54321680A69920761
:1047780007D5CA68920704D56A1E0A610022227703
:104788008A690A69520707D5CA68520704D5EA1E1A
:104798000A61002222778A690A69120707D5CA685E
:1047A800120704D5EA1F0A6100222277CA690A693A
:1047B800D20608D5CA68D20605D52A460F3A0A6134
:1047C80000222277CA690A69D20772D0CA68D2075A
:1047D8006FD00D61CA688243CA600A6A504F3A4274
:1047E80006D10A6A4F4B1A4202D10A6882430A600C
:1047F8003D23E0544C4A914244D04C4A12689142BD
:104808004BD04C4A914253D0494A126891424FD0FA
:10481800494EB1424AD0494EB14249D1EA210291AA
:104828000192002200924649029E8A5344498A8591
:10483800019AD6688643D660434E42498E664349FC
:10484800434E8E60166A3E4206D1166A354F3E4286
:1048580002D1166886431660354EF05415610099EA
:104868005162F15C012923D10221314EF154D16802
:104878000143D16037498A4240DC81078A4243D0EC
:1048880036493FE0EA212E4A50522E49354B8B6675
:1048980090852E48344981600AE0294802218185A3
:1048A8002A48C26800200121904701E02F4908707A
:1048B80021680869000605D5C868000602D528469B
:1048C8007F3808610869C00505D5C868000602D5A3
:1048D8002846FF3808610869400605D5C8684006BB
:1048E80002D528463F3808610869800604D5C8689B
:1048F800800601D51F3D0D6103B0F0BD0D498A4208
:1049080002D015498A4207D19368154919400629EA
:10491800CED003049942CBD0116801431160C7E798
:10492800111100004404000000100040381300205A
:1049380000150020004001400048014000440140AB
:10494800600E0020B010002005000020A8110020F3
:1049580025BD0008FF2B0140002C01400004004049
:10496800070001002D0200209DBE000870110020E4
:1049780070B53C22825C012A01D1022070BD02463A
:104988003C320223537000688368474C1C408460A3
:104998000B683F2B19DD5F2B1EDD602B41D00124F6
:1049A8006503AB4255D0702B79D1FF231B02846875
:1049B8009C434B688D68C9681D43090229432143FC
:1049C800816083687721194368E01F2B1EDC002B68
:1049D80020D0102B1ED062E0402B4AD0502B5ED145
:1049E800036A046A0125AC4304628469F025AC4378
:1049F800CD682D01254385610A24A34349681943DD
:104A08000162836829491940573147E0202B01D0BA
:104A1800302B44D18168254C0C402343072119438E
:104A28003CE0036A1024A34303620F231B03846939
:104A38009C43CB681B032343046A8361A0239C43E4
:104A4800496809012143016283681849194067319F
:104A580024E0FF231B0285689D434B688E68C96864
:104A68001E430902314329438160A3038168194326
:104A780014E0036A046A0125AC4304628469F025E2
:104A8800AC43CD682D01254385610A24A3434968B9
:104A98001943016283680549194047318160002044
:104AA80010700121517070BD8800CEFF88FFCFFFC4
:104AB800F0B583B0E24D2E683068E24A0240A8683B
:104AC8002969014368690843E9690843104330606C
:104AD80003200190000372688243E8681043706005
:104AE800D94A00239642184600D0286AAC69044384
:104AF800B068D64F07402743B760F06A0F24A04339
:104B08006F6A3843F062D248864212DDD148864245
:104B180016D096425CD0D048864210D1D148C06C9D
:104B28008007000FD04B1B58D04C964202970BD1F0
:104B38005CE0CA4886424FD0C948864200D010235C
:104B4800CA4C9642029751D00127F80381421FD1DF
:104B5800082B00D965E15B007B449B885B009F4480
:104B6800080060012F0160017400600160016001AC
:104B78008100C0484468BB480068800A1C21014085
:104B8800BD4840581F210140CC4000D018E147E102
:104B9800082B00D945E15B007B449B885B009F4460
:104BA800080040012F01400163004001400140011D
:104BB8007000B0484468AB480068800A1C21014076
:104BC800AD4840581F210140CC4000D018E127E1F2
:104BD800A448C06C000A01E0A248C06C0C23034042
:104BE800A148C358A14C96420297ADD10127082B82
:104BF80000D916E15B00C0467B449B885B009F445C
:104C080008001001B6001001170010011001100172
:104C1800B4009848446893480068800A1C21014001
:104C2800954840581F210140CC4000D09FE0F7E054
:104C38008C4B18688006400F25D019683820014031
:104C480008298B4A25D1144691E0864B19688906B4
:104C5800490F3CD01A6838210A40082A844A42D1B0
:104C68001446ADE00446ABE07E4B19688906490F4F
:104C780033D01A6838210A40082A7D4A52D114468E
:104C8800BEE00446BCE0083B18688004400FC440FE
:104C98006DE019680140102963D1586801990840EE
:104CA800032800D0224658684006400F411C104691
:104CB8001C4607F0BFFB61684904490E4843616818
:104CC800490F491C07F0B6FB040050D1A8E0083B87
:104CD80018688004400FC44072E0083B18688004DC
:104CE800400FC4408CE01B680B40102B5CD15D4B1F
:104CF800586801990840032800D0224658684006A1
:104D0800400F411C10461C4607F094FB616849049B
:104D1800490E48436168490F491C07F08BFB0400A2
:104D28004ED17DE01B680B40102B5DD14D4B586870
:104D380001990840032800D0224658684006400FD1
:104D4800411C10461C4607F075FB61684904490E72
:104D580048436168490F491C07F06CFB04004FD1B8
:104D68005EE019680140202963D10120C40302983C
:104D780040004249095A204607F05CFB6A680199DD
:104D8800514388424DD3110388424AD8010E540832
:104D9800000200230019594107F070FB39494118F6
:104DA800394A91423BD33CE02E4B1A680A40202AEC
:104DB800044605D018680840182831D17D2004021F
:104DC800029840002D49095A204607F033FB40005D
:104DD80069684A08101807F02DFB2949014020D0BE
:104DE8000007400F08431AE01E4B1A680A40202AA1
:104DF800044605D018680840182811D17D200402FF
:104E0800029840001D49095A204607F013FB6968BB
:104E18004A08101807F00EFB80B2102801D3F06082
:104E280000270020286768671848A866384603B036
:104E3800F0BD196801401829F2D17D20040296E7D7
:104E480020100020F369FFCF00800040FFF4FF111D
:104E5800FF4B0040004C0040003801400044004037
:104E68000048004008100240BCC700080024F400B5
:104E780000127A00E40500209CC7000812CB000845
:104E8800F0FF000000FDFFFF00FD0F000100010022
:104E980030B53448816ACA070CD18A0714D44A0746
:104EA8001CD40A0724D4CA062CD48A0634D44A0649
:104EB8003CD44CE00122520403685C689443C26A03
:104EC80022435A608A07EAD50122120403685C6803
:104ED8009443026B22435A604A07E2D501229204A6
:104EE80003685C689443426B22435A600A07DAD528
:104EF8000122D20303685C689443826B22435A60A0
:104F0800CA06D2D50122120303689C689443C26B77
:104F180022439A608A06CAD50122520303689C6814
:104F28009443026C22439A604A0610D50122130565
:104F3800026854689C43456C2C4354609D4206D1DA
:104F480003235B0554689C43836C23435360090621
:104F580007D50121C904026853688B43C06C184304
:084F6800506030BD2010002054
:104F7000F0B502462E480568EC69144000209442C2
:104F800000D1F0BD0124E6022A4F03E0EB69134093
:104F90009342F6D07B685B1A5B0E25D12B685B07CA
:104FA000F4D5EB693342F1D02E62EFF3108084F335
:104FB00010880D2149011E4D2A6813688B43136028
:104FC00080F31088EFF3108084F3108829688A68D2
:104FD000A2438A6080F3108884202021295028462B
:104FE0008C30294688311AE0EFF3108084F3108862
:104FF0000D2149010E4D2A6813688B43136080F31D
:105000001088EFF3108084F3108829688A68A2431F
:105010008A6080F3108828468830294684318022AF
:105020000023AB5420220A6002600320F0BDC0467A
:0850300020100020A81100204F
:1050380070B58421415821291AD1014656318A8AEE
:10504800002A15D0174B02E0521E140410D00C8809
:10505800002C0ED00468E5692D06F5D5056D2E885F
:105068001E40A662AC1C04650C88641E0C80EBE72D
:1050780070BDEFF31081012282F31088D305046814
:10508800A5689D43A56081F31088EFF3108182F332
:1050980010880068026840231343036081F3108876
:0850A80070BDC046FF010000CD
:1050B00030B58421415821290FD1014656310A8843
:1050C000002A0BD0026D1388104C1C4003689C62B0
:1050D000921C02650888401E088030BDEFF31081E5
:1050E000012282F3108803681C688025AC431C6091
:1050F00081F31088EFF3108182F310880068026852
:1051000040231343036081F3108830BDFF0100008A
:10511000F0B587B00268D169146895688823C358D0
:10512000222B00D09FE0059507465E372022009293
:105130007A89002A00D19CE0009A114000D198E0C1
:105140000546883579880491012205991140059119
:10515000069211020C400397019402E0890600D4E4
:1051600087E00168496A049A1140826D117039889C
:10517000491E3980816D491C81650668F1694A07BD
:1051800036D067426741CB07069B00D03B46002BD9
:1051900004D1012333626F681F436F60059B5F4238
:1051A0005F418B07069B00D53B46002B05D10223B0
:1051B00033626B6804271F436F60059B5F425F414A
:1051C000002A069A0CD53A000CD1042232626A6891
:1051D000022313436B606A68002A039F06D107E02D
:1051E000002AF2D06A68002A039F01D000226A6078
:1051F0003A88002AB2D1EFF31083012282F310889B
:10520000160207683C68B4433C60039F83F3108830
:10521000EFF31083029382F310880468A6682B468C
:10522000254D2E401D46A660019C029B83F31088ED
:10523000009B2B6000260667C36E012B8ED1C666CD
:10524000EFF3108382F310880468266810229643D7
:105250002660019C83F310880668F369DB0600D49E
:105260007CE732627AE7906908210143916107B0D7
:10527000F0BD39880029FAD07A899142F7D2EFF34C
:105280001081012282F310880B4B5B1C0468A56817
:105290001D40A56081F3108808490167EFF3108174
:1052A00082F3108800680268009B1A43026081F351
:1052B000108807B0F0BDC046FEFFFFEF77CA0008B8
:1052C000F0B587B00268D169146895688823C3581F
:1052D000222B00D09FE0059507465E3720220092E2
:1052E0007A89002A00D19CE0009A114000D198E010
:1052F0000546883579880491012205991140059168
:10530000069211020C400397019402E0890600D432
:1053100087E00668716A049A1140826D11803988AD
:10532000491E3980911C8165F1694A0736D0674270
:105330006741CB07069B00D03B46002B04D10123DD
:1053400033626F681F436F60059B5F425F418B074D
:10535000069B00D53B46002B05D1022333626B68C8
:1053600004271F436F60059B5F425F41002A069A36
:105370000CD53A000CD1042232626A68022313432E
:105380006B606A68002A039F06D107E0002AF2D00A
:105390006A68002A039F01D000226A603A88002AC6
:1053A000B4D1EFF31083012282F31088160207684C
:1053B0003C68B4433C60039F83F31088EFF3108391
:1053C000029382F310880468A66803462846264D97
:1053D0002E4005461846A660019C029B83F3108868
:1053E000009B2B6000260667C36E012B8ED1C6661C
:1053F000EFF3108382F31088046826681022964326
:105400002660019C83F310880668F369DB0600D4EC
:105410007CE732627AE7906908210143916107B025
:10542000F0BD39880029FAD07A899142F7D2EFF39A
:105430001081012282F310880B4B5B1C0468A56865
:105440001D40A56081F3108808490167EFF31081C2
:1054500082F3108800680268009B1A43026081F39F
:10546000108807B0F0BDC046FEFFFFEF01C900087D
:10547000F0B589B01546074601260791914204967A
:105480001DD31C4602260846294606F0D7FFA8422F
:1054900014D3294606F0D2FFA8420CD3294606F0C1
:1054A000CDFFA84209D3294606F0C8FF361DA84201
:1054B000EAD2761E02E0761C00E0B61C23460F9866
:1054C0000E9C03939E4200D81E4604990140002C76
:1054D0000595049133D0002931D1800703D42025CC
:1054E000002B09D002E03025002B05D0202503E059
:1054F000641EF868002822D4002C20D0A6421ED2B8
:105500007A68B968481C904202D99142F0D108E00B
:105510003A685554B860F968491CF9607A68904255
:10552000E6D13968386907F0C7F8B968884202D10E
:105530000020B860DCE70020C043F860641EF86813
:105540000890002800D5AFE0069702960127059D38
:10555000079E0194039C012C0DD96F43601E012806
:1055600011D96F43A01E012826D96F43E01E0128E0
:1055700024D9241F1CE03046394606F05FFFA842BC
:105580001ED36F4300E004463046394606F056FF0E
:10559000A84215D36F433046394606F04FFFA84264
:1055A0000ED36F433046394606F048FFA84207D372
:1055B0006F43012CDFD9D0E70446ECE70446F1E75E
:1055C0000698856807963046394606F037FF044648
:1055D000069B58686A1C824208D92A46089982426A
:1055E0000FD015460891002919D528E03248005DF2
:1055F000196848559A60D868411CD9605868824239
:10560000EFD11E461968186907F056F8B568A84228
:1056100011D10025B560F168089100290FD47C43B1
:10562000079E361B3846059C214606F007FFA74219
:105630000746C7D203E00020C0430890F0600498FA
:105640000028029F069C01982ED0002806D12BE04E
:105650001546089808900028304625D4461E8642F4
:1056600022D2874220D260686A1C824203D92A462D
:105670008242EDD10AE0206820214155A260E06815
:10568000401C0890E06060688242E1D12168206996
:1056900007F012F8A168884208D10025A560E068EB
:1056A000089000283046D9D509B0F0BD0020C0438D
:0C56B000E06009B0F0BDC046A0D20008C8
:1056BC0082B0F0B5FFB0FFB091B0FFAC2C340D460A
:1056CC00674868440260674868440360FFA8543028
:1056DC00099000226448684402606448684402608F
:1056EC00634819306349694408600AA82060E26085
:1056FC00079407E02346FFF7B5FE079CE268002AF3
:10570C0000D577E229786D1C25290BD00029079C40
:10571C0000D166E26268A368581C90422BD9934270
:10572C00EBD131E00692002729780A46233A0D2A5C
:10573C0014D802207A441279520097440B0F0F0FA1
:10574C000F0F0F0F0D0F090F0F0607436D1CEBE723
:10575C000120FAE70820F8E70420F6E70920C04307
:10576C000A463A3A0024824219D226462A462E2963
:10577C002CD0154631E02268D154A060E168491C58
:10578C00E16062689042B8D12168206906F08EFF12
:10579C00A168884200D02DE20020A060ADE7002671
:1057AC000A2256437618303E69780B463A3B8342C0
:1057BC0000D28CE072435618303EAA1CA9780B46D6
:1057CC003A3B83421546EBD22E29D2D15378194657
:1057DC003A39814200D385E0551C2878FB210246DA
:1057EC000A40682A60D1687802460A40682A00D0CC
:1057FC0072E0A87802460A40682A00D0A6E0E87851
:10580C0001402D1D6829E8D001465839202950D86F
:10581C004900C0467944898849008F442E002D00E8
:10582C002D002D002D002D002D002D002D002D0004
:10583C002D0038009D002D002D002D002D002D0079
:10584C002D002D002D002D002D002D00C1002D0050
:10585C002D00CD002D00F9002D002D002E00C0468E
:10586C005004000054040000380400003004000010
:10587C00E70300002C0400003FE70998011D099183
:10588C00016800960197FFA82C30102232E7099B83
:10589C00181D0990079C6268A168481C904212D898
:1058AC001A6823685A5468E76D1C01465839202938
:1058BC00AED9252800D020E7079C6268A168481C57
:1058CC00904200D8B2E0914200D016E75CE76A1C27
:1058DC002E2900D17AE74CE7AD1C01465839202916
:1058EC00E7D895E7511D089100240A225443E41887
:1058FC00303C0899CD1E0146287803463A3B8B4232
:10590C0000D26AE754432418303C0898851E2B7843
:10591C0018463A38884200D25FE75443E418303CCA
:10592C000898451E2B7818463A38884200D254E71E
:10593C006243D418303C0898021D037818463A3854
:10594C00884208460892D0D2151F46E7ED1C014646
:10595C0058392029ADD85BE70998011D09910168D8
:10596C00C817049141400A1A0A2A5BD30423642AFB
:10597C00A5495FD3A348824200D8C7E08A425AD3D4
:10598C0010460893059206F053FD089B1B1D9F497A
:10599C00059A8A420246EAD8DB1EA3424DD94DE055
:1059AC000998011D099101680020082300930190BA
:1059BC00FFA82C3010229EE60998011D099104685D
:1059CC00079E069F0EE03168306906F06FFEB168E5
:1059DC00884200D00EE10020B060F768641C002FF4
:1059EC0000D58AE62178002900D186E67268B36872
:1059FC00581C904202D99342F0D1E4E73268D1545A
:105A0C00B060F1684F1CF76072689042E6D1DAE73B
:105A1C000998011D0991016800960197FFA82C3087
:105A2C000A2267E60123A34207D907E0226825234F
:105A3C005354A2E69B1EA34200D82346002E04D04A
:105A4C000498002803D4002002E0002105E0012086
:105A5C000421394089080143711A0220384003900F
:105A6C00079E089301D0002C03D0F80701D1002920
:105A7C0024D10498002851D4780776D50591726802
:105A8C00B168481C904234D991425ED00698059971
:105A9C000690002869D530E63168306906F006FEBC
:105AAC00B168884200D0A5E00020B060F068069094
:105ABC00069800280599089B00D51EE6481E8842CA
:105ACC0028D28B4226D20590079E7268B168481C7A
:105ADC00904202D99142EBD1DEE732682023535435
:105AEC00B060F168491C0691F16072689042DFD198
:105AFC00D2E732682B235354089BB060F168491CE1
:105B0C000691F160726890421FD0BFE75B1EA34202
:105B1C0093D993E7079E04980028ADD50591726838
:105B2C00B168481C904201D9084609E032682D231F
:105B3C005354089BB060F168491C0691F16072687F
:105B4C000499494204919042A0D13168306906F021
:105B5C00ADFDB16888424DD10020B060F068089B63
:105B6C0005990690002800D5C7E50398002805D0B4
:105B7C0001203840204301D1002917D10091019711
:105B8C00FFA82C300A220499B4E53168306906F07C
:105B9C008DFDB16888422DD10020B060F068069070
:105BAC00089B06980028059900D5A6E5481E884252
:105BBC00E4D28B42E2D205907268B168481C9042E4
:105BCC0002D99142EDD1E0E7326830235354089B5F
:105BDC00B060F168491C0691F16072689042E0D1A6
:105BEC00D3E7002A06D0A268002A03D000200AA915
:105BFC0006F05CFD7FB07FB011B0F0BC01BC02B010
:105C0C000047C046E7030000102700009F860100F4
:105C1C00F0B587B0414F3868002808D538460C38A5
:105C2C003F4901603F490160386800285BD4012579
:105C3C006E023C46143C2068B04320600220019068
:105C4C0003900695384800680006400E801E0590AB
:105C5C0003A802A9FEF790F8E907002839D10091B2
:105C6C00354632480CC83248FDF7CEFF03260028D3
:105C7C0001962CD12D488268C3682D480830FDF759
:105C8C00C3FF002823D129480269436928481030F2
:105C9C00FDF7BAFF00281AD124488269C369244849
:105CAC001830FDF7B1FF002811D12048026A436A71
:105CBC001F482030FDF7A8FF002808D11B48826A36
:105CCC00C36A1B482830FDF79FFF00280ED02E46D4
:105CDC000099206830432060386808433860386881
:105CEC00019807B0F0BD012007B0F0BD0F48026B62
:105CFC00436B0F483030FDF787FF00282E46009984
:105D0C00E7D1206830432060386808433860386831
:105D1C00410F0420884307B0F0BDC0461420024058
:105D2C0023016745AB89EFCDE075FF1FC00600204E
:045D3C0000F001086A
:105D400010B566490A78664802704A7842708A78C7
:105D50008270CA78C2700A7902714A7942718A796E
:105D60008271CA79C2710A7A02724A7A42728A7A56
:105D70008272CA7AC2720A7B02734A7B42738A7B3E
:105D80008273CA7BC2730A7C02744A7C42748A7C26
:105D90008274CA7CC2740A7D02754A7D42758A7D0E
:105DA0008275CA7DC2750A7E02764A7E42768A7EF6
:105DB0008276CA7EC2760A7F02774A7F42778A7FDE
:105DC0008277C97FC177474A11782023C15451781F
:105DD0002123C15491782223C154D1782323C15463
:105DE00011792423C154537925240355937926240A
:105DF0000355D37927240355137A28240355537A5E
:105E000029240355937A2A240355D37A2B24035546
:105E1000137B2C240355537B2D240355937B2E2475
:105E20000355D37B2F240355137C30240355537C17
:105E300031240355937C32240355D37C33240355FA
:105E4000137D34240355537D35240355937D362427
:105E50000355D27D3723C2540368234AD3821B0CD7
:105E6000138383885383C38893830389D3834389AC
:105E7000138583895387438A9387838AD387C38A09
:105E800042241353038B44241353438B462413534C
:105E9000838B48241353C38B4A241353C3894C2444
:105EA0001353038A4E241353038C104C2380002B6E
:105EB00002D050230124D452036B9360828D382A80
:105EC00004D1C08D002803D0032010BD022010BDD6
:105ED0006539481E8141880010BDC04600F00108A8
:105EE000C006002020F00108600E00207411002080
:105EF000F0B587B0314F3868002808D538460C38DF
:105F00002F4901602F4901603868002825D40126F7
:105F1000710201913D46143D28688843286002249F
:105F200003940696284800680006400E401E05901F
:105F300003A802A9FDF726FF0221F407019E00280D
:105F400024D12248826A0746C36A2148FDF762FECF
:105F50000321002804D0194F18E0012007B0F0BD3C
:105F600000913A6B7B6B1A480830FDF753FE00280E
:105F700002D0124F009909E0BA6BFB6B1448103045
:105F8000FDF748FE00280D4F009909D028683043DE
:105F900028603868204338603868084607B0F0BD8C
:105FA0002868304328603868204338603868400FDC
:105FB00004218143084607B0F0BDC04614200240CA
:105FC00023016745AB89EFCDE075FF1FC0070020B7
:045FD00000F80108CC
:105FD400B0B505460A49002006F086FB09490020B1
:105FE40006F082FB0849002006F07EFB00202946CB
:105FF40006F07AFB0549002006F076FBB0BDC046EA
:10600400B0D200085ED000083DC800082CD00008BB
:1060140070B50D4606460A49002006F065FB0020CF
:10602400314606F061FB0749002006F05DFB0020C5
:10603400294606F059FB0449002006F055FB70BDC3
:0C604400C0D200083DC800082CD00008A5
:1060500000B5D3B04424E74E01273755A7204100AF
:106060002C914E39E44A10681B91084310607D2042
:106070001590C100E1484068369106F0DFF9401EF6
:10608000010E3A0732920322249295070029DC4B35
:1060900030D1DC494860DC4A1068DC4E304028438F
:1060A0001060002088600720086010683040D14EE2
:1060B000D7491831014311603771186C384318649F
:1060C000186C384041904198D86B32990843D86396
:1060D000D86B084041904198CE480168B9430160AF
:1060E000016802220A430260CB49EC313038026871
:1060F0000A430260219524984002C84D294614396C
:106100000A688243012358022A9010180860BB488D
:1061100041683B93980239902868400500D589E092
:10612000B74B9868D968249A8A433821309108403F
:1061300010250146349569408A18514251413B9AD5
:10614000920333920828186837942DD000292BD158
:10615000B349C91F084318603B984004B1494A68D5
:106160001B68034220D14B689B1A642BA44B00D9B7
:1061700093E11B68034217D14B689B1A642BA04B19
:1061800000D98AE11B6803420ED14B689B1A642B2D
:106190009B4B00D981E11B68034205D14B689B1AD8
:1061A000642B974BDCD978E1954DA9683098014074
:1061B0000A4634984240EB680320034002245C40C6
:1061C0001219534253412A68002963D0002B61D130
:1061D0000721C9028A43C00210182A4610601068BD
:1061E0001B99084310608F4841681268399B1A4216
:1061F00061D14268521A022A814A00D94DE11268DF
:106200001A4258D14268521A022A7D4A00D944E102
:1062100012681A424FD14268521A022A784A00D9AB
:106220003BE112681A4246D14268521A022A744A65
:10623000DBD932E1062048437B4906F0FFF8022112
:10624000081A032800D16BE7821E514251412A6887
:10625000399B1A423A4600D00A46002A00D05FE72E
:10626000421E514251412A681A423A4600D00A461B
:10627000002A00D054E7414241412A681A423A4676
:1062800000D00A46002A00D04AE7001D29681942BA
:10629000D7D145E77F2212022C4663689343339A95
:1062A0001343636000290FD0544840683579002DAE
:1062B0001BD12C461BE07F200002514B59688143C3
:1062C00033980143596034E00721C90222688A43A8
:1062D000C0021018206020688004410F5348C84055
:1062E000464948603579002DE3D0494C1834369939
:1062F00006F0A4F8401E45498842414B00D9CCE045
:10630000404A5060404800683146404E3040219E2F
:1063100030430E463C490860002090600720106022
:10632000002D00D1B9E00868384A104020430860C9
:1063300037719868309908401828186E0CD1986801
:106340003099084010282CD1D86839490140394883
:10635000814200D0A1E0B4E0012108431866314831
:1063600041681A6E9207EAD44268521A022A00D98A
:1063700093E01A6E9207E2D44268521A022A00D9B8
:106380008BE01A6E9207DAD44268521A022A00D9B8
:1063900083E01A6E9207D2D44268521A022AE0D9D8
:1063A0007BE0012001061A688A431A6040061D49F5
:1063B0004A681B6803423FD04B689B1A022B104B64
:1063C0006BD81B68034237D04B689B1A022B0C4BCF
:1063D00063D81B6803422FD04B689B1A022B084BD3
:1063E0005BD81B68034227D04B689B1A022B044BD7
:1063F000DFD952E02C11002000200240E4050020EB
:106400000010024010E000E020ED00E0FFFFFF0080
:10641000E8FFFF7F300001401405000014700040C9
:1064200007000100A811002040420F000024F400E2
:10643000737F3EEE03100222FA4CE268FA4B1340DF
:10644000FA4A9A18E260FA4A521C236813432360FE
:10645000E268329B1A43E2604A68F24B1B680342CF
:106460002FD14B689B1A022B17D8EE4B1B680342A7
:1064700027D14B689B1A022B0FD8EA4B1B680342AB
:106480001FD14B689B1A022B07D8E64B1B680342AF
:1064900017D14B689B1A022BDFD9E649002006F082
:1064A00025F9E549002006F021F9E449002006F02D
:1064B0001DF9E349002006F019F9E249002006F031
:1064C00015F938973B98C0033A90DF4800684007B9
:1064D000800F00D16EE107263003D24B996801434B
:1064E00099600F2109029A688A439A6019688901A4
:1064F00000D524E1CF49002006F0F8F8CE4900206D
:1065000006F0F4F8CD49002006F0F0F8CC49002060
:1065100006F0ECF8CB49002006F0E8F83B9DE804D3
:10652000C04A11680143116000244594506B042156
:1065300008435063506B1E9108404E904E98506B2C
:10654000202108435063506B2E9108404E904E9886
:10655000506B28435063506B28404E904E98506BC0
:10656000022108435063506B359108404E904E987D
:10657000506B082108435063506B2F9108404E9098
:106580004E986803B1491090886133988862B0488A
:106590001F278761AF48056044944394429524982F
:1065A0004003419041AE08463146FDF709FD449451
:1065B000439442953A984190A4483146FDF700FD36
:1065C00044944394429513974197A14F103F384606
:1065D0003146FDF7F5FC43954294FF201D900002E3
:1065E0002690419038463146FDF7EAFC43944294A8
:1065F00009200F900002209041900520119007077C
:1066000038463146FDF7DCFC43954294C02041906A
:106610008E483146FDF7D4FC439542943A98419018
:106620001C9738463146FDF7CBFC44944394429581
:106630004195884F283F38463146FDF7C1FC4395C8
:1066400042940C202D90419038463146FDF7B8FC1D
:10665000744EB06B2F462843B063249800037E4DE0
:1066600023902862FB02802140227C48183011C50B
:106670003398286025926A602891A9602A98E8607A
:1066800029932B6136946C61B06B384041904198EE
:10669000083D2846FDF748FA002813D06549002038
:1066A00006F024F86449002006F020F86349002031
:1066B00006F01CF86249002006F018F86149002035
:1066C00006F014F8664A1068664908403399084392
:1066D000106065492A9808603C20644F2B903C5418
:1066E0002C203B9D1F903D54FC6428032790386369
:1066F0007D633598B8637C62BC62381D04770620E0
:106700001290F861BD763C836A05A807584E3E603A
:1067100031907860BC60FC6022923A612F98786179
:106720003E943D943C943F94B86D0028349C00D135
:10673000A4E0B0683299084200D11CE144E11A4655
:1067400091680223359319430525A943916049496E
:106750004C68494A334B9F68309B1F40102F00D133
:10676000F0E14F683F1B974200D9C3E62D4B9F686D
:10677000309B1F40102F00D1E4E14F683F1B974230
:1067800000D9B7E6274B9F68309B1F40102F00D1E0
:10679000D8E14F683F1B974200D9ABE6214B9F6879
:1067A000309B1F40102F00D1CCE14F683F1B974218
:1067B000D0D99FE6244A1068022101430520814375
:1067C00011602C4841682C4A1F4B1C6807231C4051
:1067D000022C00D17FE64468641A944200D989E60D
:1067E000194C24681C40022C00D174E64468641AD9
:1067F000944200D97EE6144C24681C40022C00D13F
:1068000069E64468641A944200D973E60E4C246821
:106810001C40022C00D15EE643685B1A9342D3D938
:1068200068E6C046001002408C80C11103100222AD
:10683000FFFFFF00C0D200085ED000083DC800087E
:106840002DCD00082CD00008002002400008005088
:1068500010040050280C0050801200200400024058
:1068600008E400E0FF00FFFF00E100E01C12002050
:1068700000240140A8110020881300000025529533
:10688000519541AE301D302105F05EFF33984190A7
:106890003046FDF7D3FC002813D0F349002005F063
:1068A00025FFF249002005F021FFF149002005F005
:1068B0001DFFF049002005F019FFEF49002005F009
:1068C00015FF01200105ED4B1A6C0A431A641A6C7E
:1068D0000A4040924099596B01435963596B0140FA
:1068E0004091509503204F90CF204E9040984EA954
:1068F0001C98FDF765FBE24F239838620520E149BB
:10690000091D39607860BD60FD60289838611B986A
:1069100078613998B8612E98F8613846FDF704F926
:10692000002813D0D049002005F0E0FECF49002018
:1069300005F0DCFECE49002005F0D8FECD49002050
:1069400005F0D4FECC49002005F0D0FECE48B86258
:1069500007650746CD4A50681D9988435060CC486A
:106960002799016054203D54FD653E683B9DB06809
:106970003299084228D1B068C64901403298014393
:10698000B160C5484068C54905F058FD4000801C0D
:106990003F903F98002817D03F98401E3F903F9867
:1069A000002811D03F98401E3F903F9800280BD000
:1069B0003F98401E3F903F98002805D03F98401ECA
:1069C0003F903F980028E7D1B0683299084006D13F
:1069D000B96D2143B965F96D01220A43FA65B168C1
:1069E0001E9A1140BA6D22405118EA4323920029A1
:1069F000B96D6CD1812252009143891CB965B1688F
:106A0000C907369931D1F168182291437A68BB6879
:106A10000B43F360219B1340F96C19432B9BFB5CE8
:106A2000012B07D13B6C19437B6C0B43BD6C1D43A1
:106A30000121294333699A4D1D400D4335610123DE
:106A4000DD07AA4211D00325AD07AA420DD09B074E
:106A50009A420AD00F239B041A40924B5B1E924D20
:106A60002F681F40BA18884F2A603B6B002B279A6B
:106A700000D100223B7E9B037D7E3C46EF031F43FB
:106A8000A57E6B033B43E7681F4317432369002B35
:106A9000229A02DA854A17321A4017437A4C1F9A13
:106AA000A25C52003A432E9FE75D012F12D1002DC8
:106AB00000D1B5E0744CA56D2E9F3D43A565E56DF5
:106AC00001272F43E765656A002D07D10CE02143BC
:106AD000B96506E16C4C656A002D05D02C9F7237B4
:106AE0003D401543A26A2A43F568714F2F40174372
:106AF000F76035696F4F2F400F4337617169072584
:106B0000A943656B0D43756171697025A943A56B38
:106B10002D010D437561002B274648D00121490501
:106B20008B42349C3B9D00D08EE0396E0F230B408E
:106B30000F2BB36A7DD0F0250D40F02D79D123992C
:106B40000E397EE05C4B1C683440032C5B4F35D320
:106B50001C68359F3C43594FAC431C604B68564CF6
:106B600024683440022C29D04C68E41A944200D99D
:106B7000C0E4514C24683440022C1FD04C68E41A05
:106B8000944200D9B6E44C4C24683440022C15D011
:106B90004C68E41A944200D9ACE4474C2468344071
:106BA000022C0BD04C68E41A9442D8D9A2E4239961
:106BB0000E39B36A0B43B362349C44E02F4B99689F
:106BC0008143996098688006400F01D100F0E8FE8B
:106BD0009868309A10400828394801D100F0E5FE45
:106BE00099681140102901D001F072F9D968032287
:106BF0000A40032A00D03348D9684906490F491C86
:106C000005F01CFC1D49C9684904490E48431B494D
:106C1000C968490F491C05F011FC184B00F0C5FE6E
:106C2000294DED1F2A43184C656A002D00D055E709
:106C30005AE7FB699B001C331C251D40239B0E3B20
:106C4000AB400B43B3623B9DF168204B0B4093423A
:106C50003ED10021F965B96D01220A4302218A4320
:106C6000BA6500283DD050E0C0D200085ED00008D0
:106C70003DC800082DCD00082CD0000800100240AF
:106C8000DC120020040002401C12002008E400E096
:106C900000E100E0E8FFFF6FE4050020400D030085
:106CA00002FCFF1F0000C4FF08270140E8FFFF7F30
:106CB0001902FEFF02FCFFDF002002402C11002021
:106CC00000127A000024F40007000100E7FF3F8370
:106CD000B86D204302218843B865F86D0121014356
:106CE000F965DC49002005F001FDDB49002005F0D5
:106CF000FDFCDA49002005F0F9FCD949002005F037
:106D0000F5FCD849002005F0F1FCD7483E90369FAD
:106D10003D973C953CA8FCF73FFB002813D0CD499C
:106D2000002005F0E3FCCC49002005F0DFFCCB4956
:106D3000002005F0DBFCCA49002005F0D7FCC9495A
:106D4000002005F0D3FC3E971E983D90C7483C902C
:106D50003CA8FCF721FB002813D0BE49002005F019
:106D6000C5FCBD49002005F0C1FCBC49002005F070
:106D7000BDFCBB49002005F0B9FCBA49002005F074
:106D8000B5FC2F983D90BA483C903CA8FCF704FB1A
:106D9000002813D0AF49002005F0A8FCAE49002020
:106DA00005F0A4FCAD49002005F0A0FCAC49002092
:106DB00005F09CFCAB49002005F098FC2D983D9017
:106DC000AC483C903CA8FCF7E7FA002813D0A14956
:106DD000002005F08BFCA049002005F087FC9F49AE
:106DE000002005F083FC9E49002005F07FFC9D49B2
:106DF000002005F07BFC3D949F483C903CA8FCF7AC
:106E0000CBFA002813D09349002005F06FFC92497B
:106E1000002005F06BFC9149002005F067FC9049CB
:106E2000002005F063FC8F49002005F05FFC142072
:106E30003D9092483C903CA8FCF7AEFA002813D055
:106E40008449002005F052FC8349002005F04EFCE7
:106E50008249002005F04AFC8149002005F046FCEB
:106E60008049002005F042FC854C86482762676215
:106E7000A762E121490203C427992160676039991B
:106E8000A1602D99E160276167618426083CA159C2
:106E9000002904D12898275405F038FA20682425C1
:106EA0003296A55101683B9A91430160FDF704FEBB
:106EB00001281F952DD0A06A002801D0FDF7ECFF16
:106EC00020688168339A114381603B9BD9038268B3
:106ED0008A43826001686C4A0A4002600168194373
:106EE00001608C21675069494E680168090706D521
:106EF00022983146FEF73CF800280AD12068006845
:106F0000400767D53B9880053146FEF731F80028E9
:106F100060D05049002005F0E9FB4F49002005F002
:106F2000E5FB4E49002005F0E1FB4D49002005F04E
:106F3000DDFB4C49002005F0D9FB289AA05C012814
:106F400050D100254349284605F0D0FB4249284648
:106F500005F0CCFB4149284605F0C8FB40492846CE
:106F600005F0C4FB3F49002005F0C0FB289AA05C57
:106F7000012800D090E03749284605F0B7FB364994
:106F8000284605F0B3FB3549284605F0AFFB3449E8
:106F9000284605F0ABFB3349002005F0A7FB289AF3
:106FA000A05C012801D000F0F5FC2A49002005F082
:106FB0009DFB2949002005F099FB2849002005F098
:106FC00095FB2749002005F091FB2649002005F09C
:106FD0008DFBA2E02E993298215088202150289ACA
:106FE000A754E766329825502668336830683B9F7F
:106FF000B84330607807401EB1680140B160606EF0
:1070000022900028384617D0B568B068400F204954
:10701000095C204A105CC0001C4605F00FFA0746C8
:1070200028011F9D400F1A49095C1A4A105CC000D4
:1070300005F004FA2346289A6821114C60526A2010
:1070400027523698A05433602E9B32982350229FAB
:1070500027E0C046C0D200085ED000083DC8000846
:107060002DCD00082CD0000804FFFF07020000040B
:10707000040000080800000C8000001C40000018FC
:107080002010002000380140FFFF00FCA811002064
:1070900098D2000890D20008676E26682E9B1F9D2C
:1070A0003298255030683B9030680125A843306005
:1070B00007204006B1688143B160002F284614D0F4
:1070C000B768B068400FF84C215CF84A105CC0000B
:1070D00005F0B4F905463801400F215CF34A105C15
:1070E000C00005F0ABF9289A2E9B6821F04C605245
:1070F0006A2025523B983060329963501F98369F22
:107100006050A75430680D463168012291433160C8
:1071100051078843306063516766E64E0124346648
:107120000721B164349DF56437657765B7653246EC
:1071300040321D9802309080DF480346083B33649C
:10714000527F002A359B0DD15C22DA4B9F54DB4ADB
:10715000926B279B1A43D94EB263B26B1A40359B90
:107160004192419A5D22D34EB354C16001682943D4
:107170001D462F9B994301608760016860239943F6
:1071800001600168289B99432B460160B454CC48A8
:1071900030614997489747974697307D002828D116
:1071A000C44847755297519701256807C34AD16B68
:1071B0000143D163D16B01403C913C98506B284313
:1071C0005063506B28403C90509730204E903C9834
:1071D00003264F964EA91C98FCF7F2FEB94A906818
:1071E000B9490840B103359B014391606804B74930
:1071F0000860B0480375076204754197429743974A
:107200004497459741A83946FCF7B8FB002813D0AE
:10721000AF49002005F06AFAAE49002005F066FA91
:10722000AD49002005F062FAAC49002005F05EFA95
:10723000AB49002005F05AFA41A810211491FCF73F
:107240009DFB002813D0A249002005F04FFAA14968
:10725000002005F04BFAA049002005F047FA9F49AD
:10726000002005F043FA9E49002005F03FFA9D48B2
:107270009D4D9E4A9E49491EA4C00160476087609B
:10728000C7600C38FDF706F9002813D0904900209C
:1072900005F02CFA8F49002005F028FA8E490020CD
:1072A00005F024FA8D49002005F020FA8C490020D1
:1072B00005F01CFA8F48904A904986C005604760E7
:1072C0008760C7600C38FDF7E5F8002813D08049C7
:1072D000002005F00BFA7F49002005F007FA7E49EF
:1072E000002005F003FA7D49002005F0FFF97C49F4
:1072F000002005F0FBF9824887616322814986C03E
:10730000056047600C38FDF7C5F8002813D07049B8
:10731000002005F0EBF96F49002005F0E7F96E4910
:10732000002005F0E3F96D49002005F0DFF96C4914
:10733000002005F0DBF9744887613A46F927734964
:1073400082C0026045600838FDF7A4F8002813D019
:107350005F49002005F0CAF95E49002005F0C6F932
:107360005D49002005F0C2F95C49002005F0BEF936
:107370005B49002005F0BAF92B986349085C0128A5
:10738000634A329415D15249002005F0AFF95149B2
:10739000002005F0ABF95049002005F0A7F94F494E
:1073A000002005F0A3F94E49002005F09FF9369E14
:1073B00024E03D20359B0B5409684B68914201D174
:1073C000544A1340702293438A684B60524B99424F
:1073D00006DCA307994209D0504B994206D008E039
:1073E0004F4B994202D04A4B994202D1289B9A4373
:1073F0008A602B99444A369E56541454494CA661CF
:10740000494881C426606560083C2046FDF742F883
:107410000028354613D02E49002005F067F92D4984
:10742000002005F063F92C49002005F05FF92B4995
:10743000002005F05BF92A49002005F057F92B9848
:10744000205C012816D12249002005F04FF921497E
:10745000002005F04BF92049002005F047F91F49AD
:10746000002005F043F91E49002005F03FF9329C49
:10747000319E69E03D203599215421684B68244AAA
:10748000914201D1234A1340319E702293438A686E
:107490004B60214B994249DC329B9B0799424BD070
:1074A0001E4B994248D04AE098D2000890D200087A
:1074B00020100020C00700200830024000100240C9
:1074C0000074004008E400E0FF00FFFF00E100E07E
:1074D000C0D200085ED000083DC800082DCD0008CD
:1074E0002CD000081C140020FFF9000000480140C7
:1074F00010270000681400205FEA000000440140EB
:107500000015002000200040381300200014004027
:10751000002C01408FFF0FFFFF2B014000040040B3
:10752000004001408413002000100040C84B9942E5
:1075300002D0C84B994202D1289B9A438A602B996A
:107540006554329921540C46C348856106604560F4
:1075500085602399491CC160056144954395429516
:10756000FCF798FF002813D0BC49002005F0BEF8B6
:10757000BB49002005F0BAF8BA49002005F0B6F87A
:10758000B949002005F0B2F8B849002005F0AEF87E
:1075900027984190B04E41A93046FDF7EDF90028FB
:1075A00014D0AE49002005F0A1F8AD49002005F047
:1075B0009DF8AC49002005F099F8AB49002005F092
:1075C00095F8AA490020369D05F090F82B98305C7C
:1075D000012815D1A149002005F088F8A049002014
:1075E00005F084F89F49002005F080F89E490020AE
:1075F00005F07CF89D490020369D05F077F823E0E2
:107600003D203599315431684B68924A914201D1FD
:10761000974A1340702293438A684B60954B994276
:1076200006DCA307994209D0934B994206D008E0A3
:10763000874B994202D0874B994202D1289B9A43AB
:107640008A602B99755434548C48814A2699FF31AD
:1076500024C0056041608560C5600561449543951F
:1076600042950838FCF716FF002813D07B4900200C
:1076700005F03CF87A49002005F038F879490020F7
:1076800005F034F87849002005F030F877490020FB
:1076900005F02CF827984190784F41A93846FDF71E
:1076A0006BF9002813D06D49002005F01FF86C49D4
:1076B000002005F01BF86B49002005F017F86A4917
:1076C000002005F013F86949002005F00FF82B9809
:1076D000385C012815D16149002005F007F86049A0
:1076E000002005F003F85F49002004F0FFFF5E4929
:1076F000002004F0FBFF5D49002004F0F7FF369DF9
:1077000024E03D203599395439684B68514A9142FB
:1077100001D1574A1340702293438A684B60554BFE
:10772000994206DCA307994209D0534B994206D0EF
:1077300008E0474B994202D0464B994202D1289B20
:107740009A438A602B99369D7D543C5427464C4C75
:1077500020460830872119914900349104F0F4FF44
:10776000D22036902752474821C43D21705C012821
:1077700022910DD10220705430683E4988421CDCB1
:107780000121890788421ED03B4988421BD023E053
:107790003249002004F0AAFF3149002004F0A6FF7E
:1077A0003049002004F0A2FF3749002004F09EFF7A
:1077B0002E49002004F09AFF12E02549884202D0A9
:1077C0002449884208D1826830491140062907D0EF
:1077D00001221204914203D0016801220A4302608F
:1077E0002B49FDF76BFF00242A49204604F07EFF59
:1077F0001B49204604F07AFF1A49204604F076FF20
:107800002549204604F072FF1849002004F06EFF5D
:107810002798411E214D286817910840204940189B
:10782000112810D81F4EC046784400794000874484
:10783000080A0A0A0A0A0A0A0A0A0C0A0A0A0A0AA8
:107840004142194E37E0194E35E0194E33E0C0463B
:1078500000400140002C0140D0130020C0D200089D
:107860005ED000083DC800082DCD00082CD00008CF
:107870008FFF0FFFFF2B014000040040B4140020D5
:10788000600E0020C900010063D00008070001005D
:1078900078D00008B0D200087DD000080058014020
:1078A000AAFBFFFF82CD0008C6CD000851C8000822
:1078B000A4CD0008714E7249002004F017FF714FEB
:1078C0000020394604F012FF6F49002004F00EFF3B
:1078D0000020314604F00AFF6C49002004F006FF46
:1078E0002868030C6A493A46FDF7E8FE299D2A46B6
:1078F000383A6849FDF7E2FE2A46123A6649FDF732
:10790000DDFE6649B522FDF7D9FE209A5B32644957
:10791000FDF7D4FE634B98688006400F08D0986846
:10792000309E30400828604A2C9D0AD11F4673E0E3
:1079300018688004400F5D4AC2402C9D309E1F464F
:107940006AE098683040102818D1D8682499084017
:10795000032800D0554AD8684006400F411C104605
:107960001F4604F06BFDF9684904490E4843F96865
:10797000490F491C04F062FD02464DE09868304012
:1079800020283A9A1F4647D0B8683040182841D07E
:10799000002241E026682E9B1F983299FFF7B0FB2A
:1079A00018688004410F4148C840996889093C2201
:1079B0000A403F4989581F220A40D0403D4948604B
:1079C0003D79002D01D12C4601E03B4C183436990D
:1079D00004F034FD401E3949884201D9FEF78AFD82
:1079E00037494860374A1068344B1840219B184388
:1079F0001060002088600E60002D01D1FEF77AFD36
:107A0000114608682D4A10402043086038983871A4
:107A1000FEF784FD159802022B49FDF74FFEB8686A
:107A20008006400F3A460ED09068304008280BD0B0
:107A30009068304010281AD1D06824990840032853
:107A40004AD01A4849E010680E4C20492046FEF7FB
:107A5000E1FA1F492046FEF7DDFABFF34F8F1949BF
:107A600014391C480860BFF34F8F00BFFDE79068D2
:107A700030402028E8D09068E6E7C046E8CD00080E
:107A8000B0D200085ED000083DC800082CD0000825
:107A9000C8D200080ACE0008E4D2000840CE000890
:107AA00062CE00080010024000127A000024F400A8
:107AB0005CC70008E4050020E8FFFF7FFFFFFF0030
:107AC00010E000E020ED00E08ED0000818D30008A0
:107AD0002ACB00080400FA05FC48D1684906490F82
:107AE000491C144604F0AAFCE1684904490E4843C5
:107AF000E168490F491C04F0A1FCFB498842A3D965
:107B0000FA4B329C9C60359898601E989860F84EAD
:107B1000706871680A1A399917398A420BD27268EB
:107B2000121A8A4207D27268121A8A4203D2726803
:107B3000121A8A42EDD39C61359898611E9898611B
:107B40007068EC4F71680A1A2946A7318A420BD235
:107B50007268121A8A4207D27268121A8A4203D2D3
:107B60007268121A8A42EDD31F9AB85CE24D183D32
:107B70000128286800D1F1E1329CBC542523F95C2E
:107B8000012900D0E6E106933599F9540021F96303
:107B900039680A68A2430A60BA6CFB6C53603A6D9C
:107BA000002A02D07A6DBB6D53603A6C1C2302939D
:107BB0001A4023469340D14C22681A432260302257
:107BC00016924A60BB68CE4A102B144600D0044679
:107BD0008C60102B00D01046C8600868329A1043A1
:107BE00008600024C749204604F080FDC6492046AD
:107BF00004F07CFDC549204604F078FDC4492046C8
:107C000004F074FDC349204604F070FD0698B9499C
:107C1000085C022800D0B6E108680068800600D53C
:107C2000B8E1096C0298014035983B918840726830
:107C3000B2490B1F1E68064200D1CDE1AD4F396D30
:107C400000290ED07A6DBB6D1668334209D00E68DC
:107C50001B9F3E43A74F0E605360F96B399A114347
:107C6000F963B96CFA6C0B681A4204D04A60F96B7C
:107C70002A9A1143F9631F997C54A04A116808435A
:107C800010600698329939549E49204604F02EFD22
:107C90009D49204604F02AFD9C49204604F026FD1B
:107CA0009D49204604F022FD9A49204604F01EFD1D
:107CB000934828609948007865282ED09849204636
:107CC00004F014FD9049204604F010FD8F49204631
:107CD00004F00CFD9349204604F008FD8D49204630
:107CE00004F004FD904891490A4668C868C268C813
:107CF00068C268C868C265201F9A88543098C862F4
:107D0000886A401C8862FDF789FF89488462C462E2
:107D1000046344630487FEF7EBF8FEF711F80028CC
:107D20002C9E13D08349002004F0E0FC764900200B
:107D300004F0DCFC7549002004F0D8FC7E490020EA
:107D400004F0D4FC7349002004F0D0FC7B4A107886
:107D5000282377493B93C8540B46283350785870F2
:107D600090789870D078D8701079187150795871CF
:107D700090799871D079D871107A1872507A5872B7
:107D8000907A9872D07AD872107B1873507B58739F
:107D9000907B9873D07BD873107C1874507C587487
:107DA000907C9874D07CD874107D1875507D58756F
:107DB000907D9875D07DD875812042005888604D9F
:107DC0000992A852088D41218A0099880D92A952E2
:107DD00011210A01D9880C92A952832103914900EB
:107DE0001A896A5221210591CA0059890B92A95218
:107DF00085214A0099890A92A95243218A00D9898A
:107E00001892A95232990902401C68520893188AA4
:107E1000349968523898259F4A49C855462034906D
:107E2000285A4A213191695A414347484164E98FB0
:107E30006E20484364211A9104F000FBE853E98B5B
:107E400008042B4F294B08D00846329A10400129CC
:107E500000D010E1002800D062E1394E708B6F280D
:107E6000329900D03599652800D10021F08A328BF3
:107E70001204101804F020F85423344AD05C01286E
:107E8000329300D196E10121D154106802460832A4
:107E900083685B0700D56DE1146802231568ED0760
:107EA00000D1ACE01C4000D0A9E01468119D2C402A
:107EB000012C00D073E18468254D2C401C43846064
:107EC000249C04607C6885687CE0C04600127A00CF
:107ED0009868104020283A9800D166E598681040CC
:107EE000182854D0002060E5FF8FD0031004005004
:107EF000A81100208012002020ED00E004000240C4
:107F000000070020B0D200085ED000083DC800087D
:107F100054CB00082CD0000864D3000824F00108DA
:107F2000B8D2000830D30008CCC70008C006002033
:107F3000C0070020C0D200089FD0000800F8010848
:107F4000600E00202C110020E40500201C120020EF
:107F5000E8FFFF7F0020B8542898F863DF4900202D
:107F600004F0C4FBDE49002004F0C0FBDD49002022
:107F700004F0BCFBDC49002004F0B8FBDB49002026
:107F800004F0B4FBFEE71F980C541E9803E015980C
:107F900000020AE51B98C863D049002004F0A6FB44
:107FA000CF49002004F0A2FBCE49002004F09EFB44
:107FB000CF49002004F09AFBCC49002004F096FB46
:107FC000FEE71568ED071AD07D682D1B032DF8D349
:107FD0001568ED07F5D0E2E008263B998E401F6852
:107FE0003E4200D0F5E0C3494F68BF1A39991839AD
:107FF0008F4200D9FDE019680142F0D01EE6BE4E66
:10800000329C3155BD4C641CB56D25400D43B565A2
:1080100000243594419416681568ED07389D00D109
:10802000F2E01E4000D0EFE01568119C2540012DC4
:1080300017D18568B24C25401D438560249C04609F
:108040007E688568ED07389D04D1DDE01568ED0791
:1080500000D1D8E07D68AD1B032DF7D31568ED077F
:10806000F4D0A54CA56D149E3543A565E56D0D4373
:10807000E565359DC8E0269DFE350D4003E0A41C56
:10808000AC4200D1E6E63599996079687A68521A6F
:10809000B2420BD27A68521AB24207D27A68521AA6
:1080A000B24203D27A68521AB242EFD3359999613B
:1080B00079687A68521AB2420BD27A68521AB2427E
:1080C00007D27A68521AB24203D27A68521AB2427E
:1080D000EFD33599996079687A68521AB2420BD217
:1080E0007A68521AB24207D27A68521AB24203D25E
:1080F0007A68521AB242EFD33599996179687A68F1
:10810000521AB242BBD27A68521AB242B7D27A68D5
:10811000521AB242B3D27A68521AB242EFD3AEE7E1
:108120003598986078687968091AB1420BD27968F5
:10813000091AB14207D27968091AB14203D27968A3
:10814000091AB142EFD33598986178687968091AAD
:10815000B14200D381E67968091AB14200D37CE6C6
:108160007968091AB14200D377E67968091AB142F1
:10817000ECD372E613689B0705D41368604C234068
:10818000149C234313607B681468640700D483E65F
:108190007C68E41A032CF7D314686407F4D5002034
:1081A000554A329BD054906D149B18439065D06D06
:1081B0000843D06500244949204604F097FA48490D
:1081C000204604F093FA4749204604F08FFA4D49BF
:1081D000B4E000201F994C4C6054012002463B99AA
:1081E0008A404A4B196811431960E063069960544C
:1081F000D2E600201F99444A50542E98D0630120A3
:1082000006995054C8E6389D1668F6073A4CA66D94
:1082100042D13A4F3E4026931E43A665C368C768C5
:10822000249EB743C760364F183784683C43846048
:1082300033402193364F374E1468002C2FD5419C84
:10824000641C4194419CBC421AD81468002C26D569
:10825000419C641C4194419CBC4211D81468002C80
:108260001DD5419C641C4194419CBC4208D81468B3
:10827000002C14D5419C641C4194419CBC42DBD928
:108280001D493298359A0A54886D149A1043269ADB
:1082900090438865174F43E014990E4309E0C26884
:1082A000219C2243C260144A966D0E4326998E4348
:1082B000104F1149329A359B8B548E65002D154E07
:1082C0002ED0B4214058259908403F3000901249E3
:1082D000124A034BFDF7F2F937E0C046C0D200085E
:1082E0005ED000083DC800089ECE00082CD00008D3
:1082F000DCCE0008A81100201C120020FDFEFFFFAC
:10830000E8FFFF7FEDD0000880120020040002404B
:10831000FFF10200600E0020CCD000085CD3000802
:108320000024ED49204604F0E1F9EC49204604F030
:10833000DDF9EB49204604F0D9F9EA49002004F0C0
:10834000D5F9E949002004F0D1F9E8480069836BC8
:1083500013990B40856BFE49F94C2246FDF7AEF9A7
:10836000E802C30EFB492246FDF7A8F90124204686
:1083700002F030FCFAF7F4FE002813D0EF49002099
:1083800004F0B4F9EE49002004F0B0F9ED49002002
:1083900004F0ACF9F049002004F0A8F9EA49002003
:1083A00004F0A4F9ED4A50681E9988435060E74AEA
:1083B000507D012801D1106923E002211175106957
:1083C00002682243026002683E231340022B02D15E
:1083D000426822434260DD4A14751175E04AD21F9B
:1083E000036813430360139A520403681340620442
:1083F000934202D142680A4342600021D34A517538
:108400001475D84B00224192419041990831419115
:1084100041990A60419241904198143041904198AD
:10842000026018681B9908420E9208D018682A99B1
:10843000084204D018683999084200D0A1E01868B1
:108440001B99084208D118682A99084204D0186874
:108450003999084200D0DDE018681B99084208D01D
:1084600018682A99084204D118683999084200D03E
:10847000ACE018681B99084208D118682A9908428C
:1084800004D118683999084200D0FAE018681B999D
:1084900008421BD018682A99084217D018683999E1
:1084A000084213D11E680025AF49284604F01EF982
:1084B000A349284604F01AF9A249002004F016F94D
:1084C0002998064200D004E1A84933E018681B99B6
:1084D00008421DD118682A99084219D0186839999C
:1084E000084215D118682999084201D002F000FB12
:1084F0009F48FDF76FFD9F489F49A04AA04B7B65B1
:10850000BA65F96538669F48F8600D22002402E1DB
:108510001E6800259449284604F0E8F88849284652
:1085200004F0E4F88749002004F0E0F829980642B6
:1085300013D19549002004F0D9F88349002004F0B4
:10854000D5F88C488C498D4A8D4B7B65BA65F965A9
:1085500038668C48F8602D9ADCE08C49002004F0E5
:10856000C5F87949002004F0C1F882488249834A5D
:10857000834B7B65BA65F96538668548F8600422E7
:10858000C8E01E6800257849284604F0AFF86C4919
:10859000284604F0ABF86B49284604F0A7F8299860
:1085A00006425BD17B49002004F0A0F86649002018
:1085B00004F09CF878487949794A7A4BFB607A65EF
:1085C000B965F8653866784E2F9AA4E01D680024D6
:1085D0006549204604F08AF85949204604F086F897
:1085E0005849204604F082F8299805425ED16F4927
:1085F000204604F07BF85449204604F077F866489A
:108600006649674A674BFB607A65B965F865386605
:108610000A2280E01E6800255349284604F066F8C7
:108620004749284604F062F84649002004F05EF805
:10863000299806425CD15E49002004F057F842496F
:10864000002004F053F854485A495B4A5B4BFB60E6
:108650007A65B965F86538660F9A5BE0584900207D
:1086600004F044F83849002004F040F84A485549DD
:108670004B4A554BFB607A65B965F8653866002250
:1086800048E018682999084201D002F005FA4F48DD
:10869000FDF7A0FC40484749474A484BFB607A65D4
:1086A000B965F86538660B22002434E04849204655
:1086B00004F01CF82449204604F018F836484149D3
:1086C000374A414BFB607A65B965F8653866022226
:1086D00021E0404942E7C046C0D200085ED0000811
:1086E0003DC800083DCB00082CD00008C007002082
:1086F0000020394903F0FAFF1349002003F0F6FF88
:10870000254836492C4A364BFB607A65B965F865D1
:1087100038662246244E728532480470114B186820
:10872000279908420E9C61D13898169915462E4A11
:1087300050542A46103272855BE0C046C0D2000811
:108740005ED000083DC800082CD00008C0070020FB
:10875000FED000082BD1000880CE000804000240A3
:108760000700010010040050B0D20008BACF000882
:10877000E4CF0008FDBB00088DBB00081DBB00084E
:10878000BDBA00082DBA000894D300088DD10008A6
:1087900069BC000812CF00080100002041B60008A3
:1087A000FDB5000881B50008600E002066CF000806
:1087B0003CCF000895B8000851B80008E1B70008A0
:1087C00087CB000819B700089DB6000890CF0008B5
:1087D000DDCB000833CC0008B2CB000865B9000837
:1087E000F1B80008E40500202C1100201698F24989
:1087F0000C5418681099084206D134203899EE4D6F
:1088000029542032728502E03420EB4D2C541B9801
:10881000FBF7B0FC2A98FBF7ADFC3998FBF7AAFCF4
:108820002998FBF7A7FC2798FBF7A4FC1098FBF707
:10883000A1FC3398FBF79EFC3A98FBF79BFCDF48C2
:10884000DF49B96029656865A965E965DD4BDE48E2
:1088500058670F208004109024988005079001200D
:108860002190400704903394224613E013462A9A3D
:10887000D6480260BFF34F8FBFF36F8FEA2000210D
:108880003152D049D2488866D24802601A46D2484E
:10889000A8650B460E920FE002680A430260389802
:1088A000259960541899705A401C70527C6833980E
:1088B000844201D001F010FB3A98C8498861786879
:1088C000BD4CE066E06EA16E401A022871D3E06EE6
:1088D000A066708F596E4018E821705201B22C9832
:1088E0001C304843BE4903F089FDD821725E636E97
:1088F0009A1A8018B538C217920C821892137252C5
:108900006066EA20335A002B22D02E9E2546A45DB5
:10891000002C21D0022B26D11104B24A8A42B24E39
:10892000A54CA84D45DD217C002942D12A9BA749B1
:108930000B60BFF34F8FBFF36F8FAC490969002203
:108940008A604A6132529E48A866A248036027E0C6
:1089500000202E9960542CE03898A8550020A24E93
:108960007052686625E0032B9F4E934C954D20D1A5
:108970001104109A91421CDD217C002919D12A9BF7
:1089800092490B60BFF34F8FBFF36F8F974909690F
:1089900000228A604A6132528948A8668D48036085
:1089A000389A2598225487204000315A491C315268
:1089B0002274369D705B3746EC4E316C0C1AE01712
:1089C0008443EB483199405AEA494843000BEA494D
:1089D0004843EA4903F032FD0019810979533064B4
:1089E00088B2E74988422DD8734C207A00287E4E01
:1089F000DF4F744B40D12A9A74480260BFF34F8F07
:108A0000BFF36F8F79480069002181604161EA20DE
:108A100031526B4898666F4802601D46389B259816
:108A20002354F620315A08220A4332528320400050
:108A3000315A491C315223722B46F048A0657868A0
:108A4000A86519E0EE498842674EC94F5A4C5D4B04
:108A500012D3986DC9494018796888420CD2F62023
:108A6000315A08229143315200202072A06DE3490F
:108A7000884201D15248A0653A9858498862E14F2E
:108A8000387D002800D145E14520C10078580528EF
:108A900000D238E12F9127230146F85C26902198D7
:108AA000C0433591891E29910840D7494C1C0026A6
:108AB000D64D02E0B61CB04275D0BF19F95C6140DA
:108AC0008AB25408C90719D06C406208E10718D16E
:108AD0005408D10719D06C406208E10718D1540836
:108AE000D10719D06C406208E10718D15108D207AC
:108AF00019D069404C08C90718D118E06208E1078D
:108B0000E6D06A405408D107E5D16208E107E6D013
:108B10006A405408D107E5D16208E107E6D06A400F
:108B20005108D207E5D14C08C90700D06C403B99E9
:108B30007A5C62405108D2071AD06940B14F4A08A6
:108B4000C90719D15108D2071AD069404A08C90784
:108B500019D15108D2071AD069404A08C90719D15A
:108B60005108D2071AD069404C08C907A2D018E0B2
:108B7000A44F4A08C907E5D06A405108D207E4D19A
:108B80004A08C907E5D06A405108D207E4D14A082B
:108B9000C907E5D06A405108D207E4D14C08C9079B
:108BA00088D06C4086E73599C90721D1024D0E4E19
:108BB0003598299960E0C0462C11002031AD00089D
:108BC00001000020B010002075AD000880E100E039
:108BD0000500002000E100E07DB100080008005021
:108BE000FF0F00000000C4FF600E0020C00700203F
:108BF0003818C05C4440A0B24008E107844E1DD044
:108C000068404108C007834A1CD14808C9071DD0E5
:108C100068404108C0071CD14808C9071DD06840FA
:108C20004108C0071CD148081546C9071DD077491F
:108C3000484029994408C0071BD11CE04108C007DF
:108C4000744AE2D069404808C907E1D14108C00729
:108C5000E2D069404808C907E1D14108C007E2D025
:108C6000694048081546C907E1D129994408C00759
:108C700001D06648444035980246401C4342434177
:108C80006548415C1218521E127812025118A2B2A5
:108C90009142389900D1194600292C465F4B594F13
:108CA0002F9930D1F28B269FD31B59425941002F67
:108CB000389B00D00B46012B524F2F99574B22D196
:108CC000217D002926D11D9928313591269B7B5481
:108CD0008B218900002329917B503B997C5C102CCF
:108CE00000D157E3062C00D160E3032C00D069E3E8
:108CF0002699002900D1B4E38A4200D1B1E30B20C8
:108D0000862200F02DFC0020785038758820222122
:108D1000434A115048203590205A3299715A081A06
:108D20004142414152203152349821523798205CBF
:108D300001280F4F01D000F071FC2621308C002853
:108D400001D100F06DFC2F4A515C002901D000F0E8
:108D500067FC3449884200DDABE0411E1D2900D983
:108D60004AE3880007A108588746C046E40500206A
:108D7000A8110020B80B0000A8DE0000102700009A
:108D80000F270000298E0008FF8E00081B8F0008A7
:108D900005940008599000080594000805940008FF
:108DA000059400080594000809910008059400083E
:108DB000059400080594000805940008059400082F
:108DC000059400080594000805940008059400081F
:108DD00063910008059400080594000805940008B4
:108DE00005940008059400080594000805940008FF
:108DF00005940008059400086F910008D5AD00089F
:108E0000E12E0000240C0020FEFF000001A0000065
:108E1000600E00202C1100204B0C0020B010002010
:108E2000201000204F4F00001D46708BFD4B988096
:108E3000B08BD880F08B1881308D5881708F9881DD
:108E4000B08F5882F08F98824220305AD882F08AB0
:108E5000318B0904081818603798305A65211F9A19
:108E6000995418833098D8623498305A5883B06C2B
:108E7000D8615620305A18844C20305AD8814E2060
:108E8000305A1882986A401C9862FCF7C7FE002886
:108E900000D164E20020E94903F028FC0020E84901
:108EA00003F024FC0020E74903F020FC0020E64901
:108EB0004FE2E64988420EDCE549884200D1A6E14E
:108EC000E449884200D1A5E1E349884200D099E213
:108ED000E2485867A2E3E249884200D1A4E1E149AF
:108EE000884200D1F0E1E049884200D08AE2E06D9A
:108EF000DE49884200D091E3DD48E0658EE3708B67
:108F00006F2800D168E21C46652800D06BE2F08A29
:108F1000318B0904081800216AE21D46D548C64F66
:108F200039461CC81CC11CC81CC11CC81CC16520FA
:108F30001F9978543098F862B86A401CB862FCF700
:108F40006DFE002813D00020BC4903F0CFFB0020A9
:108F5000BB4903F0CBFB0020BA4903F0C7FB00205C
:108F6000C54903F0C3FB0020C44903F0BFFB002048
:108F7000C34908878862C86208634863FCF7B8FF82
:108F8000FCF7DEFE002813D00020AC4903F0AEFB56
:108F90000020AB4903F0AAFB0020AA4903F0A6FB7E
:108FA0000020B84903F0A2FB0020B44903F09EFB67
:108FB000B54A1078B2493B9BC8545078089B58700A
:108FC00090789870D078D87010791871507958715D
:108FD00090799871D079D871107A1872507A587245
:108FE000907A9872D07AD872107B1873507B58732D
:108FF000907B9873D07BD873107C1874507C587415
:10900000907C9874D07CD874107D1875507D5875FC
:10901000907D9875D07DD87501200002098D315260
:1090200058880999705298880D997052D8880C996F
:109030007052832040001989315258890B9970521F
:1090400098890A997052D8891899705287204000DF
:10905000198A31528D4FE0E21D4600208C4903F001
:1090600045FB0020764903F041FB0020754903F0E1
:109070003DFB0020874903F039FB00207F4903F0C6
:1090800035FB85483599405A3299715A814237D11A
:10909000708B694B9880B08BD880F08B1881308DA5
:1090A0005881708F9881B08F5882F08F98824220BB
:1090B000305AD882F08A318B090408181860379822
:1090C000305A65211F9A995418833098D862349881
:1090D000305A5883B06CD8615624305B18844C20C9
:1090E000305AD8814E20305A1882986A401C9862B3
:1090F000FCF794FD305B6849359A8852329970527A
:10910000411E8841502187E2B08DC01E80B2634964
:10911000884200D382E21698205C002800D17DE2CC
:1091200078681D4618635E4A11682398086100201C
:109130004862229BD25C012A00D03DE20222584BB9
:10914000229C1A55CB6801221343CB60554B9942A0
:1091500000DD1DE2930799424F4C00D11FE2524BB4
:109160001BE200201C4601F035FD234656E27968DB
:10917000B08DC01E80B2494A904200D34EE2186BB7
:10918000081A399A183A904200D847E24748C0680E
:10919000081A474A904200D840E24448806C081AB6
:1091A000904200D83AE21D4642480268D368012046
:1091B0008343D360136A404C234207D1399B443325
:1091C000146A1C4202D1136883431360394A229CFB
:1091D00010552963394B1968239A0A6100224A62A3
:1091E0001A5D012A01D000F057FE02221A55CA6802
:1091F0000243CA602B4A914201DD00F03CFE820727
:10920000914201D100F03DFE274A00F038FE174898
:10921000586703E2E06D1549884200D0FEE1284816
:10922000E065FBE1C0060020E06D1049884200D0F7
:10923000F4E12448E065F1E1C0060020C0D2000856
:109240005ED000083DC800082ED000086D9D0000CB
:10925000504F0000F9750000C576000075AD00089C
:109260006E9D0000E3C4000058EC000001000020E7
:10927000E9B00008CCC700084FCD00082CD000088A
:10928000C00700209FD0000800F80108A8110020A6
:10929000B0D2000838CD00082C110020FEFF0000DD
:1092A00084130020FF2B014000040040E40500204F
:1092B000102700006814002011110000381300204E
:1092C0002DAF0008C9AE00081D46708BE94B988091
:1092D000B08BD880F08B1881308D5881708F988139
:1092E000B08F5882F08F98824220305AD882F08A0C
:1092F000318B0904081818603798305A65211F9A75
:10930000995418833098D8623498305A5883B06C86
:10931000D8615620305A18844C20305AD8814E20BB
:10932000305A1882B0681863986A401C9862FCF73B
:1093300075FC002813D00020CF4903F0D7F9002096
:10934000CE4903F0D3F90020CD4903F0CFF9002036
:10935000CC4903F0CBF90020CB4903F0C7F9FCF767
:10936000EFFC00282B4600D158E10020C24903F051
:10937000BDF90020C14903F0B9F90020C04903F04C
:10938000B5F90020C14903F0B1F90020BE4903F04E
:10939000ADF942E1269900296FD08A426DD00323AE
:1093A0000B2286242198359E00F013FC2699002973
:1093B00072D08A4270D00698C000862139540220AB
:1093C0000B23BAE0359EB8192199817028994C4039
:1093D0004470249B00F001FCF08A318B09040818CA
:1093E00001211C4604E0F08A318B0904081802218F
:1093F00002F062FD234611E115998900884201D1EE
:1094000001F037FBA24A10682399016100210D4643
:109410004162229BD15C01290DD10221D154C26845
:1094200001210A43C2609B4A904257DC8A0790425E
:109430005AD0994A56E000208F4903F057F900208E
:109440008E4903F053F900208D4903F04FF90020B5
:10945000924903F04BF90020914C8B4903F046F9F7
:109460004DE044790179090209190A467E3A7C26C1
:10947000F643B24266D2032071E0427901790902D3
:109480008F1839467C397A23DE4303239024B14276
:109490006CD221981A4678E0C278817809028B183C
:1094A0008B2B44D28D2189007958C95C022903D1C4
:1094B0004721C90079580988002938D00699C90080
:1094C000129C7C525900437973547118007948708A
:1094D000359EB9190871CA7011982FE0714A9042EF
:1094E00002D0714A904207D18268704B1A40062A16
:1094F00005D00B049A4202D002680A4302603798F2
:10950000255400206A4903F0F1F800205B4903F07C
:10951000EDF800205A4903F0E9F80020654903F00E
:10952000E5F80020584903F0E1F8634B76E006982F
:10953000C0008621395402231846359E39188B55B0
:10954000431C4AE3C2788078000280180D1829462F
:109550008C398A26F643B14200D389E20220039A6D
:10956000359EB91988704A70249B36E3C178857896
:1095700028020F914618BF1938468C388A21C943F2
:10958000884200D3B4E2022221984C4F359E20E35A
:10959000444B9942424C02D0434B994209D18B68CB
:1095A000424C23403E4C062B06D01404A3423C4CB4
:1095B00002D00B6813430B60414B1968239A0A6170
:1095C00048622298185C012820D102203C4A229B44
:1095D000D054CA6801200243CA602E4A914204DC7A
:1095E0008207914207D02C4A03E02E4A914202D0D2
:1095F0002D4A914207D18A682C4B1A40062A05D081
:1096000003049A4202D00A6802430A6038982599F6
:1096100060541899705A401C70522B4600203084B8
:109620007868596B884201D1FFF740F91D465863AD
:10963000F86924491839096841403A690A40D34316
:109640003B617C690C405C407C614A402240504058
:10965000F8610240396A114302462D9B1A4033D00B
:10966000BB695B1EBB6132D11A9BBB617B6A134332
:109670007B622CE0C0060020C0D200085ED000084B
:109680003DC80008B0D400082CD000089FD00008C6
:109690001C140020FF2B014000040040D4D400081B
:1096A0002C11002000400140002C01400700010067
:1096B000B8D200086ED20008B0100020240C0020A0
:1096C00068140020280C0050209A5F32BA610B46C3
:1096D00083430822134059403962002B68D000248C
:1096E0002046FD4903F002F82046FC4902F0FEFF47
:1096F0002046FB4902F0FAFF2046FA4902F0F6FF45
:109700002046F94902F0F2FF7968B08DC01E80B2A0
:10971000F64A90422B4601D3FFF7C8F8186B081A97
:10972000399A183A904201D8FFF7C0F8F748C06854
:10973000081AF74A904201D8FFF7B8F8F348806C4E
:10974000081A904201D8FFF7B1F8F2480268D368CE
:1097500001208343D360136AEF4D2B4208D1399B1C
:109760004433166A1E42ED4E02D1136883431360E0
:10977000FA4A229D5055FC4A1163FC4B1968239A02
:109780000A614C625A5D012A00D066E102225A55F4
:10979000CA680243CA60F64A914200DD4CE1820782
:1097A000914200D14EE1F34A914200D14AE151E1A8
:1097B0007B6A1C4694430B401340594039627C62DB
:1097C000002B46D000242046DF4902F08FFF2046C0
:1097D000DE4902F08BFF2046DD4902F087FF20467C
:1097E000E54902F083FF2046DA4902F07FFFB08DA1
:1097F000C01E80B2D84988422B4601D3FFF756F8E5
:109800001698DE49085C002801D1FFF74FF8786808
:109810001863DB4A10682399016144622299515C04
:10982000012900D0A2E00221D54A229BD154C2686E
:1098300001210A43C260CE4A904200DD82E08A07DD
:10984000904200D185E02B46CA4A904200D180E088
:1098500089E00A46824304201040414039620028D2
:109860002B4601D1FFF722F800242046B64902F02A
:109870003DFF2046B54902F039FF2046B44902F0C9
:1098800035FF2046BF4902F031FF2046B14902F0C2
:109890002DFF2B46286B7968081A2C9AA632904225
:1098A00001D8FFF703F82991AC480268D368012179
:1098B0008B43D360136AAA48034208D1399B4433CF
:1098C000166A1E42A74E02D113688B431360A34A47
:1098D000229B2F91D154B28D002A2B4601D029987A
:1098E0001863B4852A9AA8480260BFF34F8FBFF36C
:1098F0006F8FEA217452A5489866A5490A60A54B66
:109900001968239A0A614C629C4AA3489065A3484F
:10991000B860A3481065229A9A5C012A73D102228A
:109920009C4B229D5A55CA682F9B1A43CA60904887
:10993000814254DC9A0791428B4D57D08D48814229
:1099400054D05CE0974A904203D02B46964A90420E
:1099500009D18268954B1A402B46062A06D00B0483
:109960009A422B4602D002680A4302607B4A106882
:109970002399016144622299515C01297F4C01D0F5
:10998000FEF78DFF0221754A229BD154C268012146
:109990000A43C260764A904208DC8A0790420ED0A1
:1099A0002B46744A90420AD0FEF776FF7D4A9042D9
:1099B00005D02B467C4A904201D0FEF76DFF8268AD
:1099C0007A4B1A402B46062A01D1FEF768FF0B049A
:1099D0009A422B4601D1FEF762FFFEF75DFF714A06
:1099E0009142614D02D0704A914208D18A686F4B12
:1099F0001A40062A07D02F9803049A4203D00A6817
:109A00002F9802430A606A4800681B9901602A99EE
:109A100001602799674801605D480160452080002A
:109A200034528920400034523C605448047404731A
:109A30002B46AC67FEF73AFF5A4A914202D05A4A87
:109A4000914207D18A68594B1A40062A05D003046F
:109A50009A4202D00A6802430A6038982599474A18
:109A600050541899705A401C70523F4BFEF71EFF1D
:109A70003599791864008C7003244C704100394A80
:109A800051182691F918269AD618777895246400EB
:109A90000F55D25C0F197A70411CA94200D3E2E144
:109AA000F178B970B178F970811CA94200D3DCE17A
:109AB0007179397131797971C11CA94200D3D6E12C
:109AC000F179B971B179F9710833001DA8423A4FA3
:109AD000D8D3DB1C359E80E0B0D200085ED00008F1
:109AE0003DC800080ED000082CD00008FEFF000082
:109AF00070001C490B184720C0002F4C205826909E
:109B00008D20800020582F3414E0C046E40500204A
:109B1000102700006814002011110000600E0020C2
:109B200021781970611E097859709B1CA41C761C41
:109B3000BE4243D2815D0029F7D00229F0D1269997
:109B400009880029ECD1F0E7B0D200085ED0000807
:109B50003DC800082CD00008FEFF0000681400205B
:109B600011110000600E0020B010002038130020FA
:109B7000FF2B01400004004089CC00082C1100207C
:109B800084130020E0D3000880E100E005000020FD
:109B900000E100E0001500207DBE000825BD0008A2
:109BA00001B5000800400140002C01400700010001
:109BB0001C12002080E200E0240C0020B94F359EEA
:109BC000B8190F99C17085701499417000241E98BE
:109BD000129B38188455801942701C462198844382
:109BE000194601402691BA19AF48471C264603E0A2
:109BF000921CB61E00D181E0107878404708C0075B
:109C00001DD0AA4847407908F8071BD14F08C8075C
:109C10001DD0A64847407908F8071BD14F08C80750
:109C20001DD0A24847407908F8071BD14808C9074A
:109C30001DD09E4948404708C0071BD11CE0790849
:109C4000F807E3D0994841404F08C807E1D17908A7
:109C5000F807E3D0954841404F08C807E1D179089B
:109C6000F807E3D0914841404808C907E1D14708C7
:109C7000C00701D08D484740517879404808C9074E
:109C80001DD08A4948404108C0071BD14808C90770
:109C90001DD0864948404108C0071BD14808C90764
:109CA0001DD0824948404108C0071BD14808C90758
:109CB0001DD07E4948404708C00799D01BE04108A5
:109CC000C007E3D0794841404808C907E1D14108BD
:109CD000C007E3D0754841404808C907E1D14108B1
:109CE000C007E3D0714841404808C907E1D147089F
:109CF000C00700D17CE76D48474079E726980028E7
:109D000002D1380A359C44E066480019359C005D54
:109D10004740B8B24008F9071DD06449484041089F
:109D2000C0071BD14808C9071DD0604948404108F9
:109D3000C0071BD14808C9071DD05C4948404108ED
:109D4000C0071BD14808C9071DD0584948404708DB
:109D5000C0071BD11CE04108C007E3D05348414075
:109D60004808C907E1D14108C007E3D04F48414046
:109D70004808C907E1D14108C007E3D04B4841403A
:109D80004808C907E1D14708C00701D04748474004
:109D9000380A444AD1180F550919487026202D99C0
:109DA00011549B1C2998135098B2414241411068AC
:109DB000024680325468202C389C00D10C46002C7E
:109DC0003B4C47D1866827998E4202D10169002910
:109DD00040D0117801293DD0014654314B800024F8
:109DE000D4600B802F49359BC918016505995160D6
:109DF000416E049B994216D127998E4203D1016985
:109E000000292C4900D02C4914704167EFF31081D0
:109E1000219A82F31088D205006883681343836017
:109E200081F3108815E027998E4203D1016900293A
:109E3000224900D0224914704167EFF31081219A22
:109E400082F3108800680268289B1A43026081F33D
:109E50001088174C002013492F9A88500875194E06
:109E6000194BFEF757FF5B1D02E0DB1D00E00933D5
:109E70000C4F359EB1E6154A914202D0144A9142E8
:109E800007D18A68134B1A40062A05D003049A4268
:109E900002D00A6802430A6038982599044A50544F
:109EA000FFF7B7FB240C0020FEFF000001A000001C
:109EB0002C11002039500008B3C90008B150000827
:109EC0001FCA0008600E0020B010002000400140B2
:109ED000002C014007000100FD48FE490160FE4DD5
:109EE000E86D8047286D8047686D8047B868804777
:109EF000A86DFA4D8047FA4A9068400090601C991E
:109F000009694904C90F4018906000D110E1686DDB
:109F1000201A4E2800D20BE16C65F249F24F3A4606
:109F2000F24BFBF7CBFBF249F24D2A463B46FBF7DF
:109F3000C5FBD820325EF049FBF7C0FBEC492A464E
:109F40003B46FBF7BBFBFC20325EEC49FBF7B6FB64
:109F5000E7492A463B46FBF7B1FBEC20325EE84975
:109F6000FBF7ACFBE2492A463B46FBF7A7FBCC20BC
:109F7000325AE449FBF7A2FBDD490D46DD4A3B4678
:109F8000FBF79CFB3698325ADF49FBF797FB2946D3
:109F9000D84A3B46FBF792FBCA20305A0028DB4ADE
:109FA00000D0DB4ADB49FBF789FBD149D14ACE4BD4
:109FB000FBF784FBC820305A0028D44A00D0D44A8A
:109FC000D549FBF77BFBCA4E3146CA4D2A46C64FE0
:109FD0003B46FBF773FBD1480069C26AD049FBF7E7
:109FE0006DFB31462A463B46FBF768FBCB480069D0
:109FF000026BCC49FBF762FB31462A463B46FBF736
:10A000005DFBEA20C84D285A0028C84A07D001281D
:10A0100001D1C74A03E00228C64A00D0C64AC74950
:10A02000FBF74CFBB24E3146B24AAF4F3B46FBF713
:10A0300045FBE220285EC2494143CA0F89148A18B1
:10A040002399083951430818C1174840431ABD499C
:10A05000FBF734FB3146A74A3B46FBF72FFBF626BE
:10A06000A85BC00703D0B849B84AFBF727FBB64F37
:10A070003946B74AFBF722FB9D499E4A9A4BFBF7AC
:10A080001DFBA948805B800703D53946AF4AFBF723
:10A0900015FB3946AF4AFBF711FB9549954A924BA0
:10A0A000FBF70CFBA048805B400703D53946A74A65
:10A0B000FBF704FB3946A84AFBF700FB8C498D4AA5
:10A0C000894BFBF7FBFA9848805B000703D53946BC
:10A0D0009E4AFBF7F3FA3946A04AFBF7EFFA8449A8
:10A0E000844A814BFBF7EAFA8F48805B800603D5F0
:10A0F0003946964AFBF7E2FA39468F4AFBF7DEFA11
:10A100007B497C4A784BFBF7D9FA954818380068A8
:10A11000C007944A04D03946934AFBF7CFFA934AD2
:10A120003946FBF7CBFA9249FBF7C8FA914F6B4DD2
:10A130002B986949085C0028199800D18E48A96BB2
:10A14000611A814200D88DE338982B99624A5054A5
:10A15000CC267548805B614DE96D3A460F1AF817B9
:10A1600087434E203390105A83494843000B83495C
:10A170004843834902F062F9C019C1086A4A915301
:10A180001646AC63E86588B2D021515A814203D2A9
:10A190003146D031504F06E0CE21715A81424E4FA8
:10A1A00002D93146CE3108803698305AD621715ABC
:10A1B000884202D93146D63105E0D421715A88420D
:10A1C00002D23146D43108806A483599405A6D49E7
:10A1D00048436D4940186D4902F010F9E221725E62
:10A1E0003E4DEB6B9A1A6A4B9A181218293AD017FF
:10A1F000C00E101840117052EA63324606B2E621D2
:10A20000515E8E4202DD1146E63105E0E421515EE9
:10A210008E4203DA1146E4310880434A118D8E42A2
:10A2200013DA4B204843642102F008F9B0423E4E55
:10A230001CDD3420385C002818D0F620315A012269
:10A24000914331520020387310E0387B0028364E9D
:10A250000CD1389B25983B54F620315A01220A43F1
:10A2600032520999705A401C70523B734148006841
:10A27000401E414241414900F620325A26239A436A
:10A280005118164A926F521E534253419A00511868
:10A290003A7C531E9A4152010A433252D820375E0B
:10A2A000002F06D4DC20315A8F420ADD37520B4B87
:10A2B00076E0E021725A784290426BDD7052074B93
:10A2C0006EE0DA20315A8F42044B69DA375267E088
:10A2D00000300040AAAA00002C110020B01000207D
:10A2E000E4050020DAD100085CD300085ED0000845
:10A2F00000D40008F8D3000808D4000814D40008DB
:10A30000DFD10008A4CC0008AFCC000824D000089E
:10A3100020D40008E8D10008F1D10008C0070020CF
:10A32000BACC0008C5CC0008600E0020D0CC0008D4
:10A33000D3CC0008D6CC0008D9CC000826D0000821
:10A3400067660000FAD10008DCCC0008F8D40008E9
:10A35000DFCC0008E2CC0008E5CC0008E8CC00081F
:10A36000280C005040D4000830D4000838D400082D
:10A370002CD00008A8110020B80B0000A8DE0000B7
:10A3800010270000140500000CE3F7FFEF060000A3
:10A39000FDFEFFFFDE21725A9042BC4B00DA705284
:10A3A000D86EF8217052186FFA217052986C196C9F
:10A3B000081AD96E0918C817000F29910818011139
:10A3C0004C23F05A88420F97269101DC0A1A00E0CC
:10A3D0000022AE4DE86C696C081A296F0E18F01750
:10A3E000000F30180711AA483399405AB8422F93EA
:10A3F00001DCC01B1218A74850431546A64901F0BE
:10A40000FDFFFC21A24A5052A048299901644664EC
:10A4100026998164C7642C98A63029904543D18F32
:10A420001646284601F0EAFFEC217052EA20305A25
:10A430009A49096D002802D1994A914207D1012811
:10A4400002D1984A914202D1974A914201D0934950
:10A450000A65964A11691269954B1B785E425E4106
:10A460004906C90F711A4B1E9941CA23884FF952E8
:10A47000D1B2C909711A3B464A1E9141C822B9524C
:10A48000401E02280BD80F980328379A66DB8948AC
:10A490001038012101607D482999016503E0012000
:10A4A00084490860379A7D4D834F985A3199695A8B
:10A4B00081429E8F18D0B04216D9764A511E8842EA
:10A4C00003D9379872490A521046319D734948534F
:10A4D00017994843114601F0B1FF6D49349A8852EB
:10A4E000495B414372484164694A3598105A6B4D43
:10A4F0002F9BE95A814214D01E2803D8139864492F
:10A50000359A8852654DE8526C4948436C4901F0D0
:10A5100095FF5F4A319950523499515A41436448EA
:10A5200041641C980069C005C00FFE2150524223AF
:10A53000D05A3399695E814200D193E16149329AE0
:10A54000895C0129359319D1B0420146514A00D99D
:10A5500009E13146B04200D307E108E100284F4D40
:10A56000554FA2DC4949086D012801DB401E0865F2
:10A5700000289AD101204F49086096E701215148EF
:10A580002F91815401688A685207414E59D44D4831
:10A59000036D1A4624325678022E2DD15678022E9B
:10A5A00000D099E01F683E680E2086433E60464812
:10A5B000851C586C066829952E40066038682F9EC9
:10A5C000B0433860186C029D284086403F4F386881
:10A5D00030433860986CDE6C46601F6D002F06D0EB
:10A5E0003868299D28403860586D9B6D4360002075
:10A5F00010702F985070304F4868149A90434860FC
:10A600008B688868C007224E39D00222134036D1A9
:10A61000886805230340012B00D089E088682C4B13
:10A62000184010438860032008607A688868C00773
:10A6300025D07868801A0328F8D38868C007F5D039
:10A6400076E08A68920705D48A6821480240149807
:10A6500002438A607A688B685B0798D57B689B1A8F
:10A66000032BF8D38B685B07F5D51648816D149AD8
:10A6700011438165C16D2F9A1143C16567E012488E
:10A68000401C144A136803405AE0C046B010002032
:10A69000600E0020B80B0000FF0F00002C110020FE
:10A6A00001B500081DB5000839B5000800080050C4
:10A6B000E4050020280C0050A811002000E204004E
:10A6C00040420F001C120020FDFEFFFF040002406C
:10A6D000E8FFFF7F741200200420D863ED4EB06DB8
:10A6E000259B1843B0654868149B98434860002038
:10A6F00010708B688868C007F94E24D0022213407E
:10A7000021D1886805230340012B11D18868F74BBC
:10A71000184010438860032008607A688868C00782
:10A7200011D07868801A0328F8D38868C007F5D05C
:10A73000EA4B986D149A104398651A465C32DB6DAB
:10A740002F9803431360C8682F9A9043C860002075
:10A75000E249329A8854359BF05AB68FB04201468E
:10A76000E04A00D8F5E6B04201D3914205D99142C2
:10A7700000D31146DA48C1520846EE49339BC8520D
:10A7800000264696F549439107994291D649419151
:10A790000127449717994843114601F04FFE459011
:10A7A00041A8F8F74FFF002813D00020E44901F03A
:10A7B0009DFF0020E34901F099FF0020E24901F0EC
:10A7C00095FF0020E14901F091FF0020E04901F0F0
:10A7D0008DFF41AD2F73E248439007984290F648B1
:10A7E00041904696E0483599405A17994843EE49BA
:10A7F00001F024FE45902846F8F724FF002813D0E6
:10A800000020CF4901F072FF0020CE4901F06EFF19
:10A810000020CD4901F06AFF0020CC4901F066FF1D
:10A820000020CB4901F062FFF8F79AFC002813D012
:10A830000020C34901F05AFF0020C24901F056FF31
:10A840000020C14901F052FF0020C94901F04EFF2C
:10A850000020BF4901F04AFFBE4A506804218843E6
:10A860005060B64FB348006E201A1A28BE4E21D34E
:10A87000B04B1C66587E400058761C9909693A9A7C
:10A8800011420FD1012108435876187F002811D1B9
:10A890003899A84A1177107D002808D0002010753B
:10A8A000BF4806E0000605D1A249087702E011750D
:10A8B000C24850650E9AA01AC14988423BD3002570
:10A8C0002846AA4901F012FF28469E4901F00EFFD2
:10A8D00028469D4901F00AFF2846BA4901F006FFC3
:10A8E00028469B4901F002FF25989249085C0128FF
:10A8F000224620D1000230589A4988620D98305A79
:10A9000088850C98305AC88583204000305A0886C4
:10A910000B98305A48860A98305A88861898305AC8
:10A92000C88687204000305A0887FBF7E1FA25984F
:10A9300080490D542246B08D022814D0012833944A
:10A94000984B01D0FDF7A6FF7A4D287B012801D155
:10A95000FDF78CFF386801283BD176489C4981651A
:10A96000904BFDF797FF7349087B01288D4B0AD167
:10A97000087E0028339401D0FDF78CFF38986D498C
:10A980000876FDF787FF087A01282BD1087E00287A
:10A99000339401D0FDF77EFF13462A9A8348026064
:10A9A000BFF34F8FBFF36F8F6E4800690021816046
:10A9B0004161EA2031526F487A49886666480260F0
:10A9C0001A46784B38985B49087679488865FDF7D0
:10A9D00061FF5849087C0128724B14D17B48886577
:10A9E000FDF758FF3868012817D15248007E00282B
:10A9F000339401D0FDF74EFF38984E4908767448DD
:10AA00008865FDF747FF986F012801D0FDF742FFE9
:10AA100048486D498165FDF73DFF4649087C01289E
:10AA200009D1087E0028339401D0FDF733FF389810
:10AA300040490876D2E7986F01280DD13D48007E45
:10AA40000028339401D0FDF725FF3898394908765E
:10AA50005D488865FDF71EFF364D297E0E92FA6827
:10AA6000204690470E9A002028764E4B3394FDF7EF
:10AA700011FF3C480069002181604161EA203152A8
:10AA8000BFF34F8F2C4914394A480860BFF34F8FEA
:10AA900000BFFDE71C12002000243449204601F0CD
:10AAA00025FE2849204601F021FE2749204601F0D5
:10AAB0001DFE3449204601F019FE2549204601F0CB
:10AAC00015FE2C482C492D4A2D4BFB607A65B96543
:10AAD000F86538660322FDF71EFEC0461C120020F2
:10AAE000600E0020B80B0000FFFF1700E8FFFF7F9B
:10AAF00000241E49204601F0F9FD1249204601F0CC
:10AB0000F5FD1149204601F0F1FD2449204601F0F0
:10AB1000EDFD0F49204601F0E9FD1B481B491C4A89
:10AB20001C4B7B65BA65F96538661B48F8600522E1
:10AB3000FDF7F1FD2C11002020ED00E0A811002010
:10AB4000C0D200085ED000083DC800082DCD000826
:10AB50002CD000080400024000E100E004000008DE
:10AB600040000018C0070020600E0020B0D200088E
:10AB700080CE00080100002065B9000851B8000827
:10AB8000F1B8000808CC0008FDBB00088DBB000828
:10AB90001DBB0008BDBA000869BC00085ECC0008F7
:10ABA00031AD0008B0100020B80B000080E100E0DB
:10ABB000D5AD00080400FA05FFFF270061B10008C9
:10ABC00081EE360058D1000811B4000825B3000802
:04ABD0003DB200088A
:10ABD400F0B582B0404F396B404A526801231C02E1
:10ABE400002806D1501A2146F431884201D802B017
:10ABF400F0BD3B480168CD689D43CD600D6A394E78
:10AC0400354206D10D6A384E354202D10D689D4356
:10AC14000D6001943D214354344CA08D002800D094
:10AC24003A630025A5855A0231480260BFF34F8F6D
:10AC3400BFF36F8FEA2025522E48B8662E48009243
:10AC44000260DF432D480268176155622C4E2D4F78
:10AC5400B7652D4F214CA7602C4F3765475C012FFA
:10AC6400019C1FD102274754D0681843D06028485C
:10AC7400824206DC9807824209D02848824206D0E4
:10AC84000DE02448824202D02348824207D19168D1
:10AC940023480840062805D01904884202D01068C9
:10ACA400184310601F48006804600099016018038D
:10ACB4001D49086010490860452080000B490D5269
:10ACC400892040000D52054805600D480574057340
:10ACD4000148856702B0F0BDB0100020A811002023
:10ACE400681400201111000044040000600E0020CC
:10ACF40080E100E00500002000E100E000150020F4
:10AD04002C1100207DBE000825BD000801B50008F7
:10AD1400FF2B014000400140002C01400004004092
:0CAD2400070001001C12002080E200E08B
:10AD300070B50F4802780A494C690A4B5B681D1BC5
:10AD4000094C002A03D0332D09D3103402E0074EFA
:10AD5000B54204D9012525606A4002704B6170BD7F
:10AD6000B0100020A811002018040050B603000005
:04AD70005811002056
:10AD740010B510480069002282604261EA200E4941
:10AD84000A520E480E4A82660E4A1368002B00D0FF
:10AD940010BD836F002B07D10C4B01241C701123B1
:10ADA4001B01CC5A641CCC520121816750680649AE
:10ADB400C86010BDC0070020600E0020B010002045
:10ADC40001000020A8110020E40500206C110020DF
:10ADD40030B586B06846C821018003AA118051802D
:10ADE400418091808180D180C1801181304901816D
:10ADF40030494B6830484268042B0AD88C68022CCE
:10AE040018D0012C08D0002C20D12C4B08241C6015
:10AE14000CE000224A6019E05B0003ACE35A0C68C2
:10AE2400141B9C4212D9254B08241C610A608A68B1
:10AE3400521C0AE05C006D462C5B0D68551BA54254
:10AE440004D90A6000225B1C4B608A601C494A6F6B
:10AE54004068042A0AD88B6F022B1BD0012B09D01F
:10AE6400002B05D1154A022313600DE0002048672A
:10AE740006B030BD520003AB9A5A0B6FC31A93420B
:10AE8400F6D90E4A022313610867886F401C88674D
:10AE940006B030BD53006C46E35A0C6F041B9C4251
:10AEA400E6D908670020521C4A67886706B030BD9F
:10AEB400C4090000B0100020A8110020180400509C
:04AEC4002C1100202D
:10AEC800F0B581B000240F4F25467E6E7B6E0E498B
:10AED8002246FAF7EFFB7519641C0C488442F4D13A
:10AEE8000146284601F0A6FA0949081A094948877F
:10AEF80002B20949FAF7DEFB08480949C16501B001
:10AF0800F0BDC046B010002012CD000850C30000AC
:10AF1800FF070000600E002059D200082C11002005
:04AF28000100002004
:10AF2C00F0B581B000255649284601F0D9FB5549AA
:10AF3C00284601F0D5FB5449284601F0D1FB534972
:10AF4C00284601F0CDFB5249284601F0C9FB514E71
:10AF5C0077687068C01B5049884224D22C4604E0A4
:10AF6C007068C01B4C4988421DD2601B4B49096F4D
:10AF7C000C18E017000F2018051149492A46FAF75A
:10AF8C0097FB70687168091A0129E9D87168091A68
:10AF9C000129E5D87168091A0129E1D87168091AE3
:10AFAC000229EFD3DCE74E203E4F385A2C1AE22010
:10AFBC00385EC72803DC6E206043642111E080B248
:10AFCC00C1084A2910D80A2141433748081880B2D1
:10AFDC00000936494143080C6E21081A4443642188
:10AFEC00204601F005FA0446A5B26E2068436421A0
:10AFFC0001F01EFA40217852FC872D4860432D4CFD
:10B00C00214601F0F5F9B88783B22B492A46FAF7A5
:10B01C004FFB2A482A4901602A49016000214160FE
:10B02C0084602949294ACA657168C26852071CD0D4
:10B03C007268521A322AF8D3C2685207F5D02449E2
:10B04C00002001F04DFB0F49002001F049FB0E4997
:10B05C00002001F045FB1F49002001F041FB0C4989
:10B06C00002001F03DFB01B0F0BD0169A14203D10C
:10B07C001949016001B0F0BD046101B0F0BDC046DA
:10B08C00B0D200085ED000083DC80008EBCC000828
:10B09C002CD00008A811002060EA0000B01000209D
:10B0AC0048D40008600E002030F8FFFF3E0A000074
:10B0BC00B80B0000FF0F000068D4000800300040FF
:10B0CC00CCCC0000555500002C11002001000020B4
:0CB0DC00C0D200082DCD0008AAAA000078
:10B0E800F0B583B000252C462F461448C66E016F74
:10B0F8000291C36E006F009011492A46FAF7DAFAF6
:10B1080034190298C7196D1C0E488542EDD10546C1
:10B118003846294601F08EF906460E4F78802046BB
:10B12800294601F087F9388082B2B3B20649FAF7A6
:10B13800C1FA06480649C16503B0F0BDB010002049
:10B1480007D2000850C3000034D200082C11002098
:08B1580001000020AC0E0020F4
:10B160000348044941650448012101607047C04615
:0CB170002C1100200100002018040050E9
:10B17C0010B52A4842682A494B68002B09D0002296
:10B18C004A6041682948426F002A0DD0002141676E
:10B19C0010BD8B68022B2AD0012B10D0002BF0D1C4
:10B1AC00214B08241C6011E0826F022A2AD0012A4C
:10B1BC0011D0002AECD11C4A0223136012E00B6858
:10B1CC00D31AC92BDDD3184B08241C610A608A687A
:10B1DC00521C8A60D5E7026F8A1AC92AD8D3124A40
:10B1EC00022313610167816F491C816710BD0B68D5
:10B1FC00D31A0C4CA342C4D90A60002201234B6021
:10B20C008A60BEE7026F8A1A064B9A42C0D9016760
:10B21C00002101224267816710BDC046A8110020A1
:10B22C00B0100020C4090000180400502C1100209C
:10B23C0030B582B06846C821018001AA11805180C6
:10B24C003049418030494B6830484268012B0AD85C
:10B25C008C68022C18D0012C08D0002C20D12C4B3F
:10B26C0008241C600CE000224A6019E05B0001AC71
:10B27C00E35A0C68141B9C4212D9254B08241C6100
:10B28C000A608A68521C0AE05C006D462C5B0D68F3
:10B29C00551BA54204D90A6000225B1C4B608A60D6
:10B2AC001C494A6F4068012A0AD88B6F022B1BD0AD
:10B2BC00012B09D0002B05D1154A022313600DE098
:10B2CC000020486702B030BD520001AB9A5A0B6F98
:10B2DC00C31A9342F6D90E4A022313610867886F8A
:10B2EC00401C886702B030BD53006C46E35A0C6FAB
:10B2FC00041B9C42E6D908670020521C4A678867E9
:10B30C0002B030BDC4090000B0100020A81100200C
:08B31C00180400502C11002060
:10B3240030B584B06846C821018002AA11805180DA
:10B33400418091803049818030494B68304842686F
:10B34400022B0AD88C68022C18D0012C08D0002CAF
:10B3540020D12C4B08241C600CE000224A6019E028
:10B364005B0002ACE35A0C68141B9C4212D9254BB7
:10B3740008241C610A608A68521C0AE05C006D465D
:10B384002C5B0D68551BA54204D90A6000225B1C86
:10B394004B608A601C494A6F4068022A0AD88B6F46
:10B3A400022B1BD0012B09D0002B05D1154A0223F7
:10B3B40013600DE00020486704B030BD520002ABBA
:10B3C4009A5A0B6FC31A9342F6D90E4A0223136199
:10B3D4000867886F401C886704B030BD53006C4612
:10B3E400E35A0C6F041B9C42E6D908670020521CE8
:10B3F4004A67886704B030BDC4090000B01000205B
:0CB40400A8110020180400502C1100209A
:10B4100030B584B06846C821018002AA11805180ED
:10B42000418091808180D1803049C18030494B6812
:10B4300030484268032B0AD88C68022C18D0012CA3
:10B4400008D0002C20D12C4B08241C600CE00022DA
:10B450004A6019E05B0002ACE35A0C68141B9C4282
:10B4600012D9254B08241C610A608A68521C0AE024
:10B470005C006D462C5B0D68551BA54204D90A6023
:10B4800000225B1C4B608A601C494A6F4068032A9B
:10B490000AD88B6F022B1BD0012B09D0002B05D1B2
:10B4A000154A022313600DE00020486704B030BD48
:10B4B000520002AB9A5A0B6FC31A9342F6D90E4A46
:10B4C000022313610867886F401C886704B030BD91
:10B4D00053006C46E35A0C6F041B9C42E6D9086784
:10B4E0000020521C4A67886704B030BDC4090000C0
:10B4F000B0100020A8110020180400502C110020CA
:10B500000348044901650448042101607047C046AE
:0CB510002C110020010000202804005035
:10B51C000348044901650448042101607047C04692
:0CB52C002C110020010000201804005029
:10B5380070B5104802780B490C690B4B5B681D1BF2
:10B548000A4C002A03D0332D0AD3103402E0084EE7
:10B55800B54205D9042525600124624002700B61BB
:10B5680070BDC046B0100020A8110020180400507B
:08B57800B6030000541100208D
:10B5800010B5002901D0022426E0154A516A431A59
:10B5900014498C6AA34221D95062134800680A7882
:10B5A000002A0AD0C0B2C409C86AA0420BD0A000C9
:10B5B000104A1018406D104A07E0FF228243D40958
:10B5C000C86AA042F3D1094A0948A300D2588A6246
:10B5D0000849C918086480470248C46210BDC046C3
:10B5E000B0100020E405002010080050F8C7000843
:0CB5F00001000020A8110020F0C7000896
:10B5FC0001204102084A1160BFF34F8FBFF36F8FD8
:10B60C000B4A10800548064A8266064801600648C7
:10B61C00064981607047C04680E100E0B010002010
:10B62C00FD01002000E100E0A811002039BE000857
:04B63C004A0F002091
:10B6400010B5012041020D4A1160BFF34F8FBFF3C7
:10B650006F8FEA220A4B00249C520A4A0A4C9466D5
:10B660000A4A11600C4908702120C000195A491C6F
:10B67000195207480749816010BDC04680E100E0CB
:10B68000600E0020B0100020D101002000E100E099
:0CB69000A811002039BE00086C11002039
:10B69C0010B5002902D00020C44326E0144A116AD8
:10B6AC00431A14490C6AA34221D91062124800684B
:10B6BC000A78002A07D0C0B2C409486AA04208DB45
:10B6CC000E4A0F480AE0FF228243D409486AA0427E
:10B6DC00F6DAA0000B4A1018406D0B4AA300D258A2
:10B6EC000A620849C918886380470248446210BD41
:10B6FC00B0100020E405002010080050F8C7000826
:0CB70C0001000020A8110020F0C7000878
:10B7180030B50120420222490A60BFF34F8FBFF3C0
:10B728006F8FEA231F490024CC521F4B1F4D9D6683
:10B738001F4B1A608C85C5431E4B1A6815615462ED
:10B748001D4C1E4DA5603D241D5D012D1FD10225F8
:10B758001D55D3680343D360194B9A4206DC83070F
:10B768009A4209D0194B9A4206D00DE0154B9A42DD
:10B7780002D0154B9A4207D19468154B2340062BEB
:10B7880005D00404A34202D0136803431360114A8E
:10B7980010702120C0000A5A521C0A5230BDC046FF
:10B7A80080E100E0600E0020B010002005000020BD
:10B7B80000E100E000150020A811002025BD0008C8
:10B7C800FF2B014000400140002C014000040040D4
:08B7D800070001006C110020C4
:10B7E00010B5002901D0022421E0124AD169431A80
:10B7F00011498C69A3421CD9D061104800680A78AD
:10B80000534253414006C40F5C40C869A04202D174
:10B810000B4A0C4804E0A0000B4A1018406D0B4A7C
:10B82000A300D2588A610849C918086380470248B2
:10B83000C46110BDB0100020E405002010080050C5
:10B84000F8C7000801000020A8110020F0C7000878
:10B8500001204102084A1160BFF34F8FBFF36F8F81
:10B860000B4A10800548064A826606480160064871
:10B87000064981607047C04680E100E0B0100020BA
:10B88000A101002000E100E0A811002039BE00085D
:04B890004A0F00203B
:10B8940010B5012041020D4A1160BFF34F8FBFF371
:10B8A4006F8FEA220A4B00249C520A4A0A4C94667F
:10B8B4000A4A11600C49087085204000195A491C35
:10B8C400195207480749816010BDC04680E100E075
:10B8D400600E0020B01000207501002000E100E09F
:0CB8E400A811002039BE00086C110020E3
:10B8F00010B5002902D00020C44321E0124A91690A
:10B90000431A12490C69A3421CD99061104800687F
:10B910000A78534253414006C40F5C404869A04234
:10B9200005DAA0000D4A1018406D0D4A01E0094AE1
:10B930000948A300D2580A610849C918886280479B
:10B940000248446110BDC046B0100020E40500204C
:10B9500010080050F8C7000801000020A8110020BE
:04B96000F0C7000824
:10B9640030B50120420222490A60BFF34F8FBFF372
:10B974006F8FEA231F490024CC521F4B1F4D9D6635
:10B984001F4B1A608C85C5431E4B1A68156154629F
:10B994001D4C1E4DA5603D241D5D012D1FD10225AA
:10B9A4001D55D3680343D360194B9A4206DC8307C1
:10B9B4009A4209D0194B9A4206D00DE0154B9A428F
:10B9C40002D0154B9A4207D19468154B2340062B9D
:10B9D40005D00404A34202D0136803431360114A40
:10B9E4001070852040000A5A521C0A5230BDC046CD
:10B9F40080E100E0600E0020B0100020050000206F
:10BA040000E100E000150020A811002025BD000879
:10BA1400FF2B014000400140002C01400004004085
:08BA2400070001006C11002075
:10BA2C00B0B5002901D004242EE0194AD16A431A7A
:10BA3C0018498C6BA34229D9D06217480268006858
:10BA4C000B785C425C415206D20F62405200002BD4
:10BA5C000BD0C0B2C0091418C86B84420CD0A00023
:10BA6C00104A1018406D104A08E0FF238343D80990
:10BA7C001418C86B8442F2D1084A0948A3000B4D34
:10BA8C00E850D2588A6380470248C463B0BDC046B0
:10BA9C00B0100020E40500201008005010C8000869
:10BAAC0001000020A811002000C80008C0070020D9
:10BABC00012041020C4A1160BFF34F8FBFF36F8F0F
:10BACC000A4A0B4B93660B4A1160104908800A48CE
:10BADC000821016009490A4A8A600A490A4A8A65AA
:10BAEC00022101607047C04680E100E0B0100020E8
:10BAFC004501002000E100E028040050A8110020BE
:10BB0C0039BE00082C110020010000204A0F002033
:10BB1C0010B50120420210490A60BFF34F8FBFF3EA
:10BB2C006F8FEA230D490324CC520D4B0D4C9C66B0
:10BB3C000D4B1A600D4A08231360022313600F4A41
:10BB4C0010702120C0000B5A5B1C0B52084809498D
:10BB5C0081600948906110BD80E100E0600E00201A
:10BB6C00B0100020CD00002000E100E028040050BF
:10BB7C00A811002039BE0008010000206C11002023
:10BB8C0030B50120420210490A60BFF34F8FBFF35A
:10BB9C006F8FEA230D490224CC520D4B0D4D9D663F
:10BBAC000D4B1A600D4A0823136014600F4A107075
:10BBBC00852040000B5A5B1C0B52094809498160D7
:10BBCC000948906130BDC04680E100E0600E002065
:10BBDC00B01000205D00002000E100E028040050BF
:10BBEC00A811002039BE0008010000206C110020B3
:10BBFC0010B501214A0210480260BFF34F8FBFF30A
:10BC0C006F8FEA230D480024C4520D4B0D4C9C66DB
:10BC1C000D4B1A60104A11702121C900435A5B1C4C
:10BC2C00435285214900435A5B1C4352074890619B
:10BC3C0007480849816010BD80E100E0600E0020DB
:10BC4C00B01000203100002000E100E041BD0008F0
:0CBC5C00A811002025BD00086C1100207C
:10BC6800B0B5002906D02C4800210170C8432349EB
:10BC78004863B0BD22498A6A821A204C236B9A42D3
:10BC88003BD988621F4801680068227853425341B3
:10BC98004906C90F59404900002A0ED0C0B2C00950
:10BCA8000D18606B85420FD01B480178012914D10B
:10BCB800A80016490818406E1BE0FF228243D009ED
:10BCC8000D18606B8542EFD1A8001149095821630E
:10BCD8000E4909180F4848660DE0002D01D00121D2
:10BCE8000170A80008490958216308490918486DD6
:10BCF8004866002800D080476563B0BDE405002091
:10BD0800B01000201008005000C80008A81100203A
:0CBD180010C80008010000206411002089
:10BD24000348044981600448102101607047C046FB
:0CBD3400A811002001000020280400508D
:10BD400030B584B06846C821018002AA11805180B4
:10BD50003449C1807D21890041808180C831918032
:10BD6000D18031494B6831484268032B0AD88C682E
:10BD7000022C18D0012C08D0002C20D12C4B0824E8
:10BD80001C600CE000224A6019E05B0002ACE35A40
:10BD90000C68141B9C4212D9254B08241C610A60B4
:10BDA0008A68521C0AE05C006D462C5B0D68551BCE
:10BDB000A54204D90A6000225B1C4B608A601D49C1
:10BDC0004A6F4068032A0AD88B6F022B1BD0012BC5
:10BDD00009D0002B05D1164A022313600DE0002084
:10BDE000486704B030BD520002AB9A5A0B6FC31AB9
:10BDF0009342F6D90E4A022313610867886F401CEC
:10BE0000886704B030BD53006C46E35A0C6F041BC6
:10BE10009C42E6D908670020521C4A67886704B034
:10BE200030BDC046C4090000B0100020A811002099
:08BE3000180400502C11002041
:10BE380070B50F4802780B49CC680B4B5B681D1B2B
:10BE48000A4C002A03D0C92D0BD3103403E019265D
:10BE58007601B54205D9102525600124624002709B
:10BE6800CB6070BDB0100020A8110020180400504D
:04BE78005011002045
:10BE7C000448082101600449044A8A6502210160D2
:10BE8C007047C046280400502C11002001000020EF
:10BE9C000348044981600448102101607047C04682
:0CBEAC00A8110020010000201804005024
:10BEB800F0B583B0C14E00230C24C14AC14D2E6099
:10BEC8007461B361F36133627362B362326070604C
:10BED80001200703002904D0012973D10324640237
:10BEE80000E08402B7603461012900D8002002977D
:10BEF8004003F06084257059002805D18020002176
:10BF0800315400F0FFF93268242001907051106814
:10BF18000127B8431060F8F7CBFD01283CD0B06A80
:10BF2800002801D0F8F7B4FFB903306882680A43E3
:10BF38008260F90382688A4382600168A24A0A40E3
:10BF48000260F90542680A434260B90602680A437A
:10BF58000260FF21090642690A40263242610168EF
:10BF6800394301608C21002474509849496802685B
:10BF7800120709D5780500970F46F8F7F5FF3946F7
:10BF8800009F002808D13068006840071ED5B80512
:10BF9800F8F7EAFF002819D000248D49204600F060
:10BFA800A1FB8C49204600F09DFB8B49204600F000
:10BFB80099FB8A49204600F095FB8949002000F04A
:10BFC80091FB0AE0B360336191D88FE7202070516C
:10BFD8008821705080203454F4667A4E306880216D
:10BFE800415C012915D17A49002000F07BFB794991
:10BFF800002000F077FB7849002000F073FB7749B8
:10C00800002000F06FFB7649002000F06BFB3068E1
:10C0180010E001468031019A4A600268136814688A
:10C02800BC4314607C07A3431360002242660A7075
:10C0380020224A60024680329168202909D181680D
:10C04800029B994202D10169002902D01178012985
:10C0580014D15F49002000F045FB6849002000F03A
:10C0680041FB5D49002000F03DFB6549002000F0E0
:10C0780039FB5B49002000F035FBFEE704465C34E1
:10C088000021C16617700368564DAB4210D05B683B
:10C098001B020DD5EFF31083019387F31088BD06BB
:10C0A800066833682B433360464E019B83F3108840
:10C0B80001673B02638001932380354627358565F8
:10C0C8008568002D0BD03E07B5420DD03E03B54222
:10C0D8000FD10569002D05D11D46FF350CE0056916
:10C0E800002D08D1FF2507E00569002D03D03F2565
:10C0F80002E0A18001E07F25A580D160222595601E
:10C10800EFF3108587F310880668B3683B43B36084
:10C1180085F310887B07456E9D42019E02D1A38955
:10C12800B34216D98368029CA342264D02D1036903
:10C13800002B18D02F4C11700467EFF3108287F38F
:10C1480010882036006803683343036082F3108840
:10C1580023E08368029CA3421A4D02D10369002B95
:10C1680003D0224C02E0224CE5E71F4C1170046713
:10C17800EFF3108287F3108803681C6834431C604F
:10C1880082F31088EFF3108287F310883B0700686A
:10C1980084681C43846082F3108826202954472031
:10C1A800C000184A2A508D208000134A2A50A984BA
:10C1B800E96129841C35A97103B0F0BD2010002065
:10C1C80000380140240C0020FFFF00FCA8110020CB
:10C1D800C0D200085ED000083DC800082DCD000878
:10C1E8002CD0000800800040C152000811510008FE
:10C1F80001C9000877CA000830060020F4D40008F6
:08C208007FD200087211002032
:10C21000032000020A490A6802404A60094D0A4C9C
:10C220002868022101225204030408401340C01868
:10C23000484068600020214600F058FAF0E7C04608
:0CC240001C1002401404005050D00008F4
:10C24C000020144900F04CFA1349002000F048FA81
:10C25C000120400411490B6802221C0413400440C5
:10C26C001B1953404B600B681C04134004401B19F2
:10C27C0053404B600B681C04134004401B19534083
:10C28C004B600B681C04134004401B1953404B605B
:10C29C00E1E7C046F8D4000800D5000814040050AB
:10C2AC0080B50248F8F75AFA80BDC04684130020C6
:10C2BC0080B50248F8F752FA80BDC046381300200A
:10C2CC0080B50248F8F74AFA80BDC0460015002038
:10C2DC0080B50248F8F742FA80BDC046B41400207D
:10C2EC0080B50248F8F73AFA80BDC04668140020C1
:10C2FC0080B50248F8F732FA80BDC0461C14002005
:10C30C00F0B595B003A808302C2100F017FA2E4890
:10C31C0000682E49884201D015B0F0BD0225049565
:10C32C000126039603A8F7F783FF002813D02849AA
:10C33C00002000F0D5F92749002000F0D1F926495A
:10C34C00002000F0CDF92549002000F0C9F924495E
:10C35C00002000F0C5F9B0032249CA680243CA6044
:10C36C00CA68024010921098086830430860086848
:10C37C0030400290149600271397129711950920BC
:10C38C0040021090029805200407019510AD20463C
:10C39C002946F7F70FFE14961397129601981190F1
:10C3AC00B002109020462946F7F704FEFF20000645
:10C3BC000D490A6882430320800710180860F006B4
:10C3CC000A49086015B0F0BD20100020003801406B
:10C3DC00C0D200085ED000083DC800082DCD000872
:10C3EC002CD000083410024018E400E000E100E01A
:10C3FC00CA1751408B1A17D0C1174A40944648406F
:10C40C00411A48081A0000E052008242FCD9002070
:10C41C0000E05208914200D3891A40419A42F8D167
:10C42C0062465040801A704710B500F075F810BD88
:10C43C000A0015D00300400800E052008242FCD9EB
:10C44C00002000E052089B1A06D340418A42F9D1E1
:10C45C00704752089B18F8D200188A42F9D17047DD
:08C46C0010B500F059F810BDF5
:10C4740038B504004D42FFF7DFFF4543611938BD6D
:10C48400002B09D1002907D110B51100FFF7F0FFE7
:10C494000A000021002310BD70B400240125ED071B
:10C4A400002B07D1002905D0834203D213000022B8
:10C4B4002C0000250026A419994200D1904212D9DB
:10C4C40092185B4103D2EE076D086408F3E7DE07B8
:10C4D4005B08520892190126F6079B1903E0DE0750
:10C4E4005B0852089219801A994103D364416D4143
:10C4F400F5D30FE024196D410AD2DE075B08520818
:10C50400921980185941F5D364416D41E7D301E094
:10C514008018594102000B002000290070BC7047AC
:08C52400002000217047C04611
:10C52C0003230F480F4A036143610F4B8261C361C0
:10C53C008023DB000362002383624362C3620266D2
:10C54C000A4A426610228266094A0367C366436739
:10C55C001178013AC1540133102BF9D17047C04600
:10C56C00780F002034C80008240800204C15002047
:04C57C004FC800089C
:10C58000F8B54746CE46C5688368040040689946BA
:10C590005B1B80B50E00170098464019934207D9DF
:10C5A00000F0CAF8ED19E560C0BCB946B046F8BD68
:10C5B0001A0000F0C1F84B463100ED19ED1A2A00BF
:0CC5C0006068414400F0B8F8EDE7C046A8
:10C5CC00F8B54746CE46002380B5884607001600CE
:10C5DC009946C56884681BE0013B5B1B641BB44235
:10C5EC0000D934009C4200D91C00786822004146D6
:10C5FC00401900F09BF82D19A144A044361BBC68CF
:10C60C00631B5A1E93415B421D40FD60002E06D0F9
:10C61C003B699D42E0D3013B1B195B1BDEE748469F
:08C62C00C0BCB946B046F8BDE0
:10C6340070B50600431C5C00E4181D4BE400E018D0
:10C644007400A419E4001B19DC6A1500012C06D03F
:10C65400022C1FD0002C10D00024200070BD9A6A38
:10C664005C6AA2421FD9013A121B2C00954200D9E0
:10C6740014002200FFF782FFEFE79A6A5E6AB24273
:10C684000CD9013A961BB542E7D82A00FFF776FF8A
:10C694002C00E2E7FFF798FF0400DEE71B6AD218DC
:10C6A400013A961BEFE71B6AD218013A121BDCE72A
:04C6B400780F0020DB
:10C6B800F8B50B4B04001B780D001600002B0CD0AE
:10C6C800EFF31087012181F3108832002900200040
:10C6D800FFF7ACFF87F31088F8BDFFF723FFEFE7FC
:04C6E800780F0020A7
:10C6EC00F8B5050008000C0000F018F80A4B06001D
:10C6FC001B78002B0CD0EFF31087012181F31088ED
:10C70C00320021002800FFF78FFF87F31088F8BD57
:0CC71C00FFF706FFEFE7C046780F002093
:10C72800411C02780130002AFBD1401A7047C046EC
:10C73800002A03D0013A8B5C8354FBD17047C04672
:10C7480000220B0011001A00002A02D0013A81547D
:04C75800FCD1704759
:10C75C0000000000000000000000000000000000CD
:10C76C0000000000000000000000000000000000BD
:10C77C0001000000020000000300000004000000A3
:10C78C00060000000700000008000000090000007F
:10C79C00000000000000000000000000000000008D
:10C7AC000100000002000000030000000400000073
:10C7BC00000000000400000002000000080000005F
:10C7CC00004B0000650001000100E80300000000C0
:10C7DC00000064008800DC05F401AA02A406200213
:04C7EC000000000049
:08C7F0000A000000B80B000074
:08C7F8000100000064000000D4
:10C800000A000000B80B0000B80B0000B80B0000D5
:10C8100001000000640000006400000064000000EB
:10C82000034C206804348047FBE7F9F711FCFEE76E
:04C8300014D5000813
:09C834005465726D696E616C00BF
:03C83D003A20009E
:10C840000000000000005454522052454747455311
:01C8500000E7
:10C851004465766963652049443A20756E6B6E6F55
:03C86100776E00EF
:02C86400FEE7ED
:02C86600FEE7EB
:02C86800FEE7E9
:02C86A00FEE7E7
:02C86C00FEE7E5
:02C86E00FEE7E3
:02C87000FEE7E1
:02C87200FEE7DF
:02C87400FEE7DD
:02C87600FEE7DB
:02C87800FEE7D9
:02C87A00FEE7D7
:02C87C00FEE7D5
:02C87E00FEE7D3
:02C88000FEE7D1
:02C88200FEE7CF
:02C88400FEE7CD
:02C88600FEE7CB
:02C88800FEE7C9
:02C88A00FEE7C7
:02C88C00FEE7C5
:02C88E00FEE7C3
:02C89000FEE7C1
:06C89200F6F715FCC3E7F8
:10C8980010B5816A8B6D8A6D5024234205D0D2066B
:10C8A80012D4096D496B884710BD012043021A4311
:10C8B8008A650A68D3681B059B0F05D18B7E002B00
:10C8C80002D113681B0700D410BD93685B0709D415
:10C8D800583153680C24A3435360FF2302330A687A
:10C8E8009A4305E08A6D202313438B65CA6D5C313A
:06C8F80002430A6010BDBE
:02C8FE00704781
:10C9000070B588214158222901680FD102465E3254
:10C910005388496A1940836D19801188491E118016
:10C92000991C81651188002905D070BD886908228D
:10C9300002438A6170BD02468832EFF31083012101
:10C9400081F310880924640105682E68A6432E60CF
:10C9500083F31088EFF3108381F310880468A568CF
:10C960008D43A56083F310882023136000220267A3
:10C97000C36E012BD9D1C266EFF3108281F3108808
:10C9800003681C6810218C431C6082F310880068C7
:0AC99000C269D206C9D5016270BD6C
:02C99A007047E4
:02C99C007047E2
:10C99E00806A816D40220A438265C16D04220A437A
:04C9AE00C2657047A7
:10C9B20030B584214158212904D1014656318A8A51
:10C9C200002A03D130BD521E1304FBD00B88002B6A
:10C9D2000CD00368DC692406F5D5046D25789D62C8
:10C9E200631C03650B885B1E0B80ECE7EFF3108181
:10C9F200012282F31088D3050468A5689D43A560CF
:10CA020081F31088EFF3108182F3108800680268C6
:0CCA120040231343036081F3108830BD03
:10CA1E0030B58421415821290DD1014656310A885D
:10CA2E00002A09D00268036D1C7894625A1C0265B4
:10CA3E000888401E088030BDEFF31081012282F37A
:10CA4E00108803681C688025AC431C6081F3108835
:10CA5E00EFF3108182F310880068026840231343BD
:08CA6E00036081F3108830BD64
:10CA760070B5882141582229016810D102465E32DC
:10CA86005388496A1940836D19701188491E1180AF
:10CA9600816D491C81651188002905D070BD8869A2
:10CAA600082202438A6170BD02468832EFF3108382
:10CAB600012181F310880924640105682E68A643C4
:10CAC6002E6083F31088EFF3108381F310880468D7
:10CAD600A5688D43A56083F3108820231360002288
:10CAE6000267C36E012BD9D1C266EFF3108281F3C0
:10CAF600108803681C6810218C431C6082F3108820
:0CCB06000068C269D206C9D5016270BD8A
:10CB1200010002000400060008000A000C001000D8
:08CB220020004000800000012A
:10CB2A00547279696E6720746F20726573746172CA
:03CB3A00742E0056
:10CB3D004144432063616C6962726174696F6E2058
:07CB4D006572726F72210096
:10CB54005374617274696E6720566563746F7220D2
:10CB64005461626C6520636F7079696E67206672C8
:10CB74006F6D20464C41534820746F2052414D2E16
:03CB84002E2E0052
:10CB87004D6F646520302069732073656C6563742D
:10CB970065642E204175746F2D7265636F6E6E65C7
:0BCBA7006374206973204F46462E0087
:10CBB2004D6F646520312069732073656C65637401
:10CBC20065642E204175746F2D7265636F6E6E659C
:0BCBD2006374206973204F46462E005C
:10CBDD004D6F646520322069732073656C656374D5
:10CBED0065642E204175746F2D7265636F6E6E6571
:0BCBFD006374206973204F46462E0031
:10CC08004D6F646520332069732073656C656374A8
:10CC180065642E204175746F2D7265636F6E6E6545
:0BCC28006374206973204F46462E0005
:10CC33004D6F646520342069732073656C6563747C
:10CC430065642E204175746F2D7265636F6E6E651A
:0BCC53006374206973204F46462E00DA
:10CC5E004D6F646520352069732073656C65637450
:10CC6E0065642E204175746F2D7265636F6E6E65EF
:0BCC7E006374206973204F46462E00AF
:10CC8900555020627574746F6E206973206C6F6ED5
:0BCC9900672D707265737365642E00D8
:0BCCA40056613A20253664206D5600D2
:0BCCAF0056623A20253664206D5600C6
:0BCCBA004441435F413A2025346400F0
:0BCCC5004441435F423A2025346400E4
:03CCD0004F5000C2
:03CCD300434C00CF
:03CCD600424100D8
:03CCD900414200D5
:03CCDC00257300BD
:03CCDF004F5400AF
:03CCE2004F4300BD
:03CCE5004F4C00B1
:03CCE8004C4200BB
:10CCEB0043757272656E742063616C6C69627261FC
:10CCFB0074696F6E2073657175656E6365207374EF
:07CD0B0061727465642E00E3
:10CD1200095B2534645D2053616D706C6564207617
:0BCD2200616C75653A202534640A003E
:0BCD2D0048414C206572726F722100BB
:10CD380053415645204C4F434B2D4B455920434FAB
:07CD48004D4D414E442E0049
:10CD4F0043616E6E6F7420726573746F72652064C9
:10CD5F00656661756C742073657474696E67732092
:10CD6F0066726F6D20464C415348206D656D6F7232
:03CD7F0079210017
:10CD82004465766963652049443A2053544D3332F1
:10CD920047304231206F722053544D333247304373
:02CDA20031005E
:10CDA4004465766963652049443A2053544D3332CF
:10CDB40047303731206F722053544D333247303867
:02CDC40031003C
:10CDC6004465766963652049443A2053544D3332AD
:10CDD60047303531206F722053544D333247303649
:02CDE60031001A
:10CDE8004465766963652049443A2053544D33328B
:10CDF80047303331206F722053544D33324730342B
:02CE08003100F7
:10CE0A004672656520737061636520666F72206380
:10CE1A006F66696775726174696F6E20696E2066E4
:10CE2A00616B6520454550524F4D3A202575206269
:06CE3A00797465730A0023
:10CE40004D41585F504F535349424C455F4449460A
:10CE5000465F544F5F4D4541535552453A20257525
:02CE60000A00C6
:10CE62004144435F4241545F435249544943414C18
:0ECE72005F564F4C544147453A2025750A0043
:10CE800043616E6E6F742073746172742041444309
:0ECE900020696E20444D41206D6F64652100C5
:10CE9E0043616E6E6F7420636F7079205665637494
:10CEAE006F72205461626C652066726F6D20464C05
:10CEBE0041534820746F2052414D2120444D412052
:0ECECE006973206E6F742072656164792100B3
:10CEDC0043616E6E6F742066696E69736820636F50
:10CEEC007079696E6720566563746F722054616245
:10CEFC006C652066726F6D20464C41534820746FF0
:06CF0C002052414D2100FE
:10CF12004D6F646520302069732073656C6563749E
:10CF220065642E204175746F2D7265636F6E6E6538
:0ACF32006374206973204F4E2E0037
:10CF3C004D6F646520312069732073656C65637473
:10CF4C0065642E204175746F2D7265636F6E6E650E
:0ACF5C006374206973204F4E2E000D
:10CF66004D6F646520322069732073656C65637448
:10CF760065642E204175746F2D7265636F6E6E65E4
:0ACF86006374206973204F4E2E00E3
:10CF90004D6F646520332069732073656C6563741D
:10CFA00065642E204175746F2D7265636F6E6E65BA
:0ACFB0006374206973204F4E2E00B9
:10CFBA004D6F646520342069732073656C656374F2
:10CFCA0065642E204175746F2D7265636F6E6E6590
:0ACFDA006374206973204F4E2E008F
:10CFE4004D6F646520352069732073656C656374C7
:10CFF40065642E204175746F2D7265636F6E6E6566
:0AD004006374206973204F4E2E0064
:10D00E00555020627574746F6E206973207072654E
:06D01E00737365642E002F
:02D024004E00BC
:06D02600523A20257300C0
:02D02C000A00F8
:10D02E0043616E6E6F742073617665206461746106
:10D03E0020696E20464C415348206D656D6F7279A4
:02D04E002100BF
:0ED050004E4D49204552524F522121210A00D7
:05D05E004D41494E00A8
:10D0630043616E6E6F742073746172742054494D02
:05D073004552322100CE
:05D078001B5B324A00C1
:10D07D0050726F6772616D20737461727465642E86
:01D08D0000A2
:10D08E0043505520467265713A20257520487A0A1C
:01D09E000091
:10D09F0043616E6E6F74207265616420636F6E669C
:10D0AF00696775726174696F6E2066726F6D204665
:0DD0BF004C415348206D656D6F7279210062
:10D0CC00257325733A204144432043616C69627295
:10D0DC006174696F6E2076616C75653A2025750AEE
:01D0EC000043
:10D0ED0043616E6E6F742073746F702041444321E1
:01D0FD000032
:10D0FE0025733A204441432043616C696272617426
:10D10E00696F6E2076616C756520666F722063683C
:0DD11E00616E6E656C20313A2025750A00A7
:10D12B0025733A204441432043616C6962726174F8
:10D13B00696F6E2076616C756520666F722063680F
:0DD14B00616E6E656C20323A2025750A0079
:10D1580049742069732074696D6520746F20736148
:10D16800766520737461746973746963616C206493
:10D1780061746120696E20466C617368206D656D0D
:05D188006F72792E001A
:10D18D00496C6C6567616C204D6F64652069732017
:10D19D0073656C65637465642E2044656661756C9A
:10D1AD0074204D6F646520342069732073656C6540
:10D1BD00637465642E204175746F2D7265636F6E97
:0DD1CD006E656374206973204F46462E0086
:05D1DA00257325730020
:09D1DF00493A2025356420410085
:09D1E8004F56503A202531730026
:09D1F1004C56503A202531730020
:0DD1FA00543A202532642E256420B04300F5
:10D20700095B2534645D2053616D706C656420761D
:10D21700616C7565733A20492B203D2025367520B2
:0DD22700202020492D203D202536750A00CD
:10D2340009094F66667365742076616C7565733A87
:10D2440020492B203D20257520202020492D203DDC
:05D254002025750A0011
:10D2590009094F66667365742076616C75653A20B5
:05D269002534640A00F9
:10D26E00556E6B6E6F776E20636F6D6D616E6421A0
:01D27E0000AF
:0DD27F005553415254206572726F722100A8
:04D28C00D130000895
:08D29000010101030701000088
:08D29800080402040801010171
:10D2A00030313233343536373839414243444546DC
:08D2B0001B5B323B33326D00C1
:08D2B8001B5B323B33336D00B8
:08D2C0001B5B323B33316D00B2
:10D2C80025733A205265766973696F6E206E756DA5
:0CD2D8006265723A2030782534580A0054
:10D2E4004672656520737061636520666F72207392
:10D2F40074617469737469637320696E2066616B09
:10D304006520454550524F4D3A2025752062797469
:04D3140065730A0033
:10D31800435055207370656564206973206E6F747F
:08D328002036344D487A210043
:10D330004669727374207374617274212057726924
:10D3400074696E672064656661756C7420636F6EC6
:0CD3500066696775726174696F6E210078
:08D35C001B5B313B33326D0015
:10D36400566563746F72205461626C6520686173E2
:10D37400206265656E20636F706965642066726FF4
:10D384006D20464C41534820746F2052414D2E006D
:10D39400496C6C6567616C204D6F6465206973200E
:10D3A40073656C65637465642E2044656661756C91
:10D3B40074204D6F646520342069732073656C6537
:10D3C400637465642E204175746F2D7265636F6E8E
:0CD3D4006E656374206973204F4E2E00BC
:10D3E000444F574E20627574746F6E2069732070BD
:08D3F0007265737365642E0081
:08D3F8001B5B323B33306D007A
:08D400002573207C2025730038
:0CD408005661623A20253464206D560005
:0CD414005662623A20253564206D5600F7
:10D420001B5B323B33316D591B5B313B33326D003B
:08D430001B5B313B33366D003C
:08D43800434847202D2031007C
:08D44000434847202D20300075
:10D448000909566F6C746167652D64726F702041AD
:10D4580044432076616C75653A202535642E0A00B0
:10D4680009090946696E616C20766F6C746167659D
:10D478002D64726F70204144432076616C75653A63
:10D48800202534752E2046696E616C20766F6C7489
:10D498006167652D64726F702076616C75653A20DE
:08D4A800253375206D560A00C2
:10D4B00043616E6E6F742073617665206E657720B0
:10D4C000534E20696E20464C415348206D656D6F68
:04D4D000727921004C
:10D4D40043616E6E6F742073746172742054494D8D
:10D4E400313720696E20495352206D6F64652100E5
:04D4F4004D4F440054
:08D4F8001B5B313B33316D0079
:10D50000486172646661756C74204552524F5221B5
:04D5100021210A00CB
:10D5140019FC0008C00600203800000019FC0008AF
:10D52400000700207608000019FC0008780F00208E
:10D53400E40500002BFC0008000000205CD5000876
:10D54400BB0600002BFC00080060002017DC00086C
:08D55400002000002BC80008B4
:10D55C007047C04609480069C16A0E2905D8026B9C
:10D56C0081600E2A06D8426170470F39026B8160C8
:10D57C000E2AF8D90F3A42617047C046C007002006
:10D58C0009480069C16A0E2905D8026B81600E2A10
:10D59C0006D8426170470F39026B81600E2AF8D9A8
:10D5AC000F3A42617047C046C0070020F0B51648DC
:10D5BC000069016B3A22154B9C5E154D6A6E12196F
:10D5CC00144EB242144F02DAB9421AD310E00123BE
:10D5DC000E291F4600D800276D6E2C19B44200DCB2
:10D5EC0000233B400E22D2430B4F002B00D0891856
:10D5FC004161C16AB94201D38160F0BD0F318160D4
:10D60C00F0BD0F22F3E7C046C0070020600E0020DB
:10D61C00B0100020AC060000F10F0000F0B5184867
:10D62C000069C16A3A22174B9C5E174D6A6E12193B
:10D63C00164EB242164F03DA0E2911D8002310E011
:10D64C000123B9421F4600D300276D6E2C19B4423A
:10D65C0000DC00233B400F220D4F002B05D105E0D1
:10D66C0001230E22D243002B00D089188160016B5C
:10D67C00B94201D34161F0BD0F314161F0BDC046EB
:10D68C00C0070020600E0020B010002052090000DE
:10D69C00F10F000009480069C26A09498A4205D3A2
:10D6AC00036B82608B4206D3436170470F32036B6E
:10D6BC0082608B42F8D20F3343617047C007002061
:10D6CC00F10F000009480069C16A0E2905D8026BE8
:10D6DC0081600E2A06D8426170470F39026B816057
:10D6EC000E2AF8D90F3A42617047C046C007002095
:10D6FC0009480069C26A09498A4205D3036B8260F2
:10D70C008B4206D3436170470F32036B82608B42AE
:10D71C00F8D20F3343617047C0070020F10F0000AF
:10D72C0009480069C16A0E2905D8026B81600E2A6E
:10D73C0006D8426170470F39026B81600E2AF8D906
:10D74C000F3A42617047C046C00700200948006983
:10D75C00C26A09498A4205D3036B82608B4206D3A5
:10D76C00436170470F32036B82608B42F8D20F33E8
:10D77C0043617047C0070020F10F000009480069A1
:10D78C00C26A09498A4205D3036B82608B4206D375
:10D79C00436170470F32036B82608B42F8D20F33B8
:10D7AC0043617047C0070020F10F00000248416838
:10D7BC00491C41607047C046A8110020F0B581B0EB
:10D7CC00194F3889194CA08001208503124E356001
:10D7DC00A0688047B8887989E06021610F480168AA
:10D7EC0002220A430260E0682169884200DC084694
:10D7FC0040210B4A515E884208D3216808182060EA
:10D80C000849496C884203D9606980470020206030
:10D81C00356101B0F0BDC04618080050040002404C
:10D82C00600E0020E4050020F011002010110020F3
:10D83C0011480069002181604161EA220F48815240
:10D84C0001210A030E4B1A60BFF34F8FBFF36F8F8A
:10D85C000C4A0D4B9366926F002A00D070470D4A0C
:10D86C00117041229200835A5B1C8352074801605D
:10D87C004068074988647047C0070020600E00208C
:10D88C0080E100E0B010002001000020A811002071
:10D89C00E40500206C110020F0B58BB0A1480068A5
:10D8AC00C469016801220A921207079209908768DD
:10D8BC0023070891049756D0501C384001252A02A2
:10D8CC00164620360E4006434DD00A40564256416D
:10D8DC00E2070A9A00D03246002A07D109990D6254
:10D8EC008C2290498E582E438E5008993D406A42A6
:10D8FC006A41A6070A9E00D51646002E0AD10222BE
:10D90C0009990A628C2287498E58042737438F5015
:10D91C00049F08996A426A4165070A9D04D4002D48
:10D92C0004D0002B0ED41EE01500FAD10422099964
:10D93C000A628C227B498D5802262E438E50089900
:10D94C00002B10D5421E90418A060A9A00D402463A
:10D95C00012A08D10820099908628C2271498B5838
:10D96C0003438B5008990123D8050590200514D545
:10D97C003846059A10409A060A4010180DD0D80265
:10D98C00099908628820202266490A5084200A508E
:10D99C00089965480375654A8354202025460690EE
:10D9AC0005402CD03846079A10400A46069E324055
:10D9BC00024324D002934520C0005B4A13588826AA
:10D9CC00584FBE59222E12D102990E02B3420ED2DA
:10D9DC00D31809994E6A2727DE55544B0299D15416
:10D9EC0013585B1C13500B460899049F07E00999C8
:10D9FC008869082202438A610899049F029B80204F
:10DA0C0026460390064032D03846059A10400A4606
:10DA1C00039F3A4002432AD043480068842282582C
:10DA2C00212A14D1024656321788002F12D00768CB
:10DA3C000197076D02973F780092019A9762029ABC
:10DA4C00571C0765009A1088401E10800BE0006878
:10DA5C00026802E000680268039FBA430260026831
:10DA6C00402717430760304A2320000113544027F6
:10DA7C000A463A4050425041620600D50A900A9834
:10DA8C0000280ED109990868B843086084202549FC
:10DA9C00069A0A50264800220270882022240C5034
:10DAAC004A678C221F48805800282ED088242220B8
:10DABC001C490A9408510899002D09D0049D029321
:10DACC00079B2B400D46069C25401D43029B1ED1F7
:10DADC00002E1AD0049A059D2A40039C2140114324
:10DAEC0013D009990A68BA430A6084210D4A1D466D
:10DAFC001346069A5A500A99585026200A49002271
:10DB0C000A54232000010D545A670BB0F0BD09993B
:10DB1C008869082303438B610020024988500BB0AD
:10DB2C00F0BDC04620100020240C00203102000063
:10DB3C004A0C0020010000000024F400FFFFFFFF4E
:10DB4C00C0E0FFFF01000000FFFFFFFF010000002D
:10DB5C000200000001000000FFFFFFFF01000000B9
:10DB6C000200000001000000FFFFFFFF01000000A9
:10DB7C000400000000B80B00FFFFFFFFC0E0FFFF38
:10DB8C00000000000202000000000002020202027B
:10DB9C000100000000000000000000000001010175
:10DBAC000001010001000202010100000000000060
:10DBBC000000000000000000000000000000000059
:10DBCC000000000000000000000000000000000049
:10DBDC000000000000000000000000000000000039
:10DBEC000000000000000000000000000001010126
:10DBFC000100010100000001010101000000000012
:10DC0C000000000000000000000000CDCDCDCDCD07
:10DC1C00CDCDCDCDCDCDCDCDCDCDCDCDCDCDCDCD28
:10DC2C00CDCDCDCDCDCDCDCDCDCDCDCDCDCDCDCD18
:10DC3C00CDCDCDCDCDCDCDCDCDCDCDCDCDCDCDCD08
:10DC4C00CDCDCDCDCDCDCDCDCDCDCDCDCDCDCDCDF8
:0CFC0C00CDCDCDCDCDCDCDCDCDCDCD001D
:10FC1800206861680834002200E042540139FCD5AC
:02FC2800704723
:10FC2A0020686168A2680C3401E08B5C8354013A55
:04FC3A00FBD570473F
:10FC3E00FFFFFFFFFFFFFFFFFFFFFFFFFFFFFFFFC6
:10FC4E00FFFFFFFFFFFFFFFFFFFFFFFFFFFFFFFFB6
:10FC5E00FFFFFFFFFFFFFFFFFFFFFFFFFFFFFFFFA6
:10FC6E00FFFFFFFFFFFFFFFFFFFFFFFFFFFFFFFF96
:02FFFE00FFFF03
:020000040801F1
:10000000FFFFFFFFFFFFFFFFFFFFFFFFFFFFFFFF00
:10001000FFFFFFFFFFFFFFFFFFFFFFFFFFFFFFFFF0
:10002000FFFFFFFFFFFFFFFFFFFFFFFFFFFFFFFFE0
:10003000FFFFFFFFFFFFFFFFFFFFFFFFFFFFFFFFD0
:04EFFC00C4DBD31C83
:040000050800C89394
:00000001FF
